:108da400510798002e019000be0190004e009000e3
:108db400de009000020040008380480020079800f5
:108dc400310798000000eb00c08288000040eb00ef
:108dd4005ff0b7001e009000100178002e00900094
:108de400be009000a21f07000004e00003003a0048
:108df4008081eb00230f9800060037002e009000be
:108e0400be009000d0828800e18288008000eb00e0
:108e1400210f98002e0890000080fa000000060040
:108e24003200fa00500f9800620f9800730f9800f8
:108e34000040eb005ff0b7005e08900040589000df
:108e44000080fb00201798002e109000e10f5000c6
:108e540014003200ae109000e38f50000100320085
:108e64002e0037006e089000fe0890004209dd00d5
:108e7400ce00de00810071004200dd00200f98006a
:108e8400310f9800f0ff2f00f1ff20002007980019
:108e94003107980080ff2f00f1ff2000008fbe00f3
:108ea4002b003700ee08900030002000000ab800c4
:108eb4006e0890006000b9000501780000014100cf
:108ec4007e0890006300b90000014100820278002e
:108ed400240f9800350f98002e0890006140600020
:108ee400005f98002e089000be0890008100d10019
:108ef4000080d300200f9800310f9800f0ff2f005e
:108f040001002000200798003107980080ff20000e
:108f140001002000008fbe000d0037006e08900095
:108f2400fe0890000000400081804800200f980057
:108f3400310f9800f0ff2f00010020002007980057
:108f44003107980080ff2f0001002000008fbe0031
:108f54005e08900030019000c00190002e0890003f
:108f6400be089000470add004900de0000007200e0
:108f7400c908de000200400083804800000f98000a
:108f8400110f98002e089000be089000f21f2000d8
:108f940003002000000278008102780002007800bb
:108fa4008300780000016200018062006102b80061
:108fb40034179800451798003e109000ce1090008a
:108fc400c000dd0000002000301798004117980011
:108fd4003e109000ce1090006112b8003417980033
:108fe400451798003e119000ce11900002007000c9
:108ff40083807000200f9800310f980092828000c7
:10900400a38280000e0890009e089000800f5100fb
:10901400818f5900a8003a005e08900040589000e3
:10902400e34f500008003a002e08900080007800ba
:1090340080c62000008040001002be006407980033
:10904400750798003a0137005e0890004058900078
:10905400e24f500009003a002e089000800078008a
:1090640080c620000080400010007800010020002d
:1090740060079800710798002d0137005e08900082
:1090840040589000e14f500029013a002e0890000a
:109094008000780080c620000080400010407800e6
:1090a4000080fb0001002000600798007107980011
:1090b4000e5890000004e000080032006e0090009a
:1090c400fe009000cc0add004400de000080720047
:1090d400c408de0060079800710798002e0890000d
:1090e400be08900061004000e0804800f21f2000ac
:1090f400030020000002780081027800020078005a
:109104008300780000016200018062006102b800ff
:1091140054179800651798005e109000ee109000a8
:10912400c000dd000000200050179800611798006f
:109134005e109000ee1090006112b8005417980071
:10914400651798005e119000ee1190000200700007
:1091540083807000200f9800310f98002e08900033
:10916400be089000e00f5000e08f580027003a003e
:1091740056d0bf000004e0000d00320011c0b3005f
:109184006022b8006011b8005e089000f800070083
:10919400e00f5000e08f5800050032002e029000ce
:1091a400be0290000417980015179800ec003700d1
:1091b4000e0890009e08900061004000e080480086
:1091c40082c62000aa1e07000004e00009003a003d
:1091d400f0ff2f000100200090828800a182880007
:1091e4002e009000be009000001798001117980000
:1091f400db0037000e0890009e08900061004000dc
:10920400e080480090828800a18288002e089000a7
:109214008000780080c62000008040001040780064
:109224000080fb00010020004007980051079800cf
:109234000e5890000004e0000d0032004e00900033
:10924400de0090004409dd00cc01de0083017100e2
:109254004401dd006e009000fe009000000041001b
:10926400818049006007980071079800b0003700ba
:109274004e009000de0090006f0160006000b800b6
:109284000300200002007000838070004809dd00a4
:10929400c801de00830171004801dd006e0090000a
:1092a400fe009000000041008180490060079800a2
:1092b400710798009e00370056d0bf000004e000fc
:1092c4000d00320011c0b3006022b8006011b80074
:1092d4005e089000a6000700e00f5000e08f5800e1
:1092e400050032002e019000be0190000217980084
:1092f400131798009a00370082c620000e089000c9
:109304009e0890005a1e07000004e00009003a007d
:10931400f0ff2f000100200090828800a1828800c5
:109324002e029000be0290000417980015179800b2
:109334008b0037000e0890009e08900090828800f1
:10934400a18288005e08900040589000e34f5000ce
:1093540008003a002e0890008000780080c62000a3
:10936400008040001001be00620798007307980057
:109374006f0037005e08900040589000e24f5000a4
:1093840009003a002e0890008000780080c6200072
:109394000080400010007800010020006007980061
:1093a40071079800620037005e08900040589000f2
:1093b400e14f50005e003a002e08900080007800d3
:1093c40080c6200000804000104078000080fb0030
:1093d4000100200060079800710798000e58900063
:1093e4000004e000080032006e009000fe009000cf
:1093f400cc09dd004400de0000807100c408de00fa
:1094040060079800710798002e089000be0890002d
:1094140061004000e0804800f21f200003002000ab
:10942400000278008102780002007800830078004e
:1094340000016200018062006102b80074179800a4
:10944400051f98007e1090008e189000c000dd006b
:109454000000200070179800011f98007e109000f3
:109464008e1890006112b80074179800051f9800b8
:109474007e1190008e1990000200700083807000ad
:10948400200f9800310f98002e089000800078007b
:1094940080c6200000804000104078000080fb005f
:1094a4000100200040079800510798000e589000d2
:1094b4000004e0000d0032004e009000de00900039
:1094c4004409dd00cc01de00830171004401dd00ac
:1094d4006e009000fe009000000041008180490071
:1094e4006007980071079800110037004e00900043
:1094f400de0090006f0160006000b80003002000ef
:1095040002007000838070004809dd00c801de009d
:10951400830171004801dd006e009000fe009000a0
:10952400000041008180490060079800710798009d
:109534006e009000fe009000be0f5000ae8f5800e9
:10954400030039001e02be006407980075079800e6
:109554006e009000fe00900000179800111798000c
:109564000e1090009e1090000080fa00000006008b
:109574004000fa00200f9800320f9800430f980023
:10958400540f9800650f9800615f98002e089000b2
:1095940040589000e34f50000d0032002e08900018
:1095a40040589000e24f5000090032002e0890000d
:1095b40040589000e14f500005003200f0ff2f00aa
:1095c400f1ff20002017980031179800120237008d
:1095d4002e089000405890000080fb00101798005f
:1095e4009e109000e18f50000e0035001e11900077
:1095f400e20f5100080034009e119000e38f5100e7
:109604000100320007003700f0ff2f00f1ff2000b7
:10961400008fbe0003003700f0ff2f000100200080
:10962400008fbe000040eb005ff0b7006e58900062
:109634000004e000290032000040eb0020579800ad
:1096440094828000a5828000440798005507980002
:109654001700370090828000a18280008041eb00d7
:1096640082c62000711e07000004e00004003a00d6
:109674001e00be002017980031179800e60137003d
:109684002e5090000040e800205798002e089000cb
:10969400400890006101b8004e009000de00900088
:1096a400000041008180490040079800510798005c
:1096b4002e089000a05890002e50900080cf5000ab
:1096c400e4ff3e000040eb0056f0b7006011b80024
:1096d4002217980033179800cf0137002e08900006
:1096e400405890000080fb00001798008e119000f5
:1096f400e18f51000d0032000e129000e30f520072
:1097040001003200200037003e089000ce0890008f
:10971400c20add00ce00de00818072004200dd005e
:1097240060079800710798001d003700be0890007c
:1097340030002000000ab8003e0890006000b90024
:1097440005017800000141004e0890006300b90053
:1097540000014100820278006407980075079800b0
:109764006e00900061406000105798006e009000f9
:10977400fe0090008100d1000080d30060079800b3
:1097840071079800060037003e089000ce0890004c
:10979400000040008180480060079800710798002d
:1097a4002e08900030019000c00190006e009000df
:1097b400fe009000470add004900de000000720050
:1097c400c908de000200400083804800200798009a
:1097d400310798006e009000fe009000f21f2000f8
:1097e4000300200000027800810278000200780063
:1097f4008300780000016200018062006102b80009
:1098040044179800551798004e109000de109000f1
:10981400c000dd0000002000401798005117980098
:109824004e109000de1090006112b80044179800aa
:10983400551798004e119000de1190000200700040
:1098440083807000600798007107980092828000fe
:10985400a38280002e009000be009000800f510073
:10986400818f59003a00320056d0bf000004e00056
:10987400250032000040eb002057980094828000bd
:10988400a582800044079800550798001700370008
:1098940090828000a18280008041eb0082c620007b
:1098a400e21d07000004e00004003a001e00be00b0
:1098b4002017980031179800570137002e50900058
:1098c4000040e800205798002e08900040089000bf
:1098d4006101b8004e009000de00900000004100dd
:1098e4008180490040079800510798002e08900095
:1098f400a05890002e50900080cf5000e4ff3e000e
:109904000040eb0056f0b70082c620002e00900005
:10991400be009000d61c07000004e00008003a00d6
:10992400f0ff2f000100200090828800a1828800af
:109934001e01be0022179800331798003601370025
:109944002e029000be02900094828800a5828800b6
:109954002e08900040589000e34f500072003a00e7
:109964006e0090008000780080c620008080400057
:109974005e089000804878006e00900080007800b7
:1099840090c62000008340005e089000ee0890001e
:1099940002f02f000300200000027800810278000a
:1099a40002007800830078000001620001806200f8
:1099b4006102b80064179800751798006e10900043
:1099c400fe109000c000dd00000020006017980029
:1099d400711798006e109000fe1090006112b8008c
:1099e40064179800751798006e119000fe1190008e
:1099f4000200700083807000c809dd004800de00aa
:109a040000807100c808de00004b78006e009000f2
:109a140080007800a0c62000008340005e0890000b
:109a2400ee08900002002000f30f200000027800ee
:109a3400810278000200780083007800000162004f
:109a4400018062006102b800041f9800151f98008d
:109a54000e1890009e189000c000dd000000200049
:109a6400001f9800111f98000e1890009e18900077
:109a74006112b800041f9800151f98000e19900079
:109a84009e19900002007000838070004008de0080
:109a940001002000004b78006e00900080007800e8
:109aa400b0c62000008340005e089000ee089000dd
:109ab4000200200003f020000002780081027800f8
:109ac40002007800830078000001620001806200d7
:109ad4006102b800241f9800351f98002e189000ca
:109ae400be189000c000dd0000002000201f980078
:109af400311f98002e189000be1890006112b80013
:109b0400241f9800351f98002e199000be1990004c
:109b140002007000838070004808de00010020000d
:109b2400004b7800b70037002e0890004058900092
:109b3400e24f50002c003a006e0090008000780044
:109b440080c62000808040005e0890008048780035
:109b54006e0090008000780090c6200000834000d2
:109b64005e089000ee08900002f02f000300200031
:109b740000027800810278000200780083007800f7
:109b840000016200018062006102b800441f980075
:109b9400551f98004e189000de189000c000dd009c
:109ba40000002000401f9800511f98004e1890009c
:109bb400de1890006112b800441f9800551f9800e9
:109bc4004e199000de19900002007000838070002e
:109bd400c809dd004800de0000807100c808de000e
:109be400004b7800870037002e0890004058900002
:109bf400e14f500083003a006e009000800078002e
:109c040080c620000080400010427800045798006d
:109c14001e5090000004e000080032005e0890002e
:109c24006f406000c400dd000e5090006f40600083
:109c340000c0700000579800020037005e089000d2
:109c4400005798006e0090008000780080c62000c5
:109c5400008040008e529000054878006e0090000d
:109c6400fe00900061004000e0804800f21f2000e8
:109c740003002000000278008102780002007800ce
:109c84008300780000016200018062006102b80074
:109c9400641f9800751f98006e189000fe189000bd
:109ca400c000dd0000002000601f9800711f9800b4
:109cb4006e189000fe1890006112b800641f98009e
:109cc400751f98006e199000fe1990000200700034
:109cd4008380700060079800710798006e00900000
:109ce400fe009000e00f5000e08f580022003a0080
:109cf40011c0b3006022b8006011b8002e089000b3
:109d04001bfe0700e00f5000e08f580004003200f3
:109d14001e02be0024179800351798003e00370035
:109d24002e009000be00900061004000e0804800da
:109d340082c62000ce1b07000004e00008003a00a1
:109d4400f0ff2f000100200090828800a18288008b
:109d54001e00be0020179800311798002e0037000f
:109d64002e009000be00900061004000e08048009a
:109d740090828800a18288006e00900080007800a4
:109d840080c6200000804000904078000157980071
:109d94001e5090000004e000080032005e089000ad
:109da400ee0890004c09dd004400de000000710064
:109db400c408de00005798000c0037005e089000cd
:109dc400ee089000c809dd004800de000080710044
:109dd400c808de006f4160008e50900000cfb300d1
:109de40000c0600000407100005798006e009000b1
:109df4008000780080c62000008040000e52900051
:109e04000448780010c0b30056f0b7006000b800f2
:109e140020179800311798002e109000be10900063
:109e24000080fa00000006000200fa00000f78002b
:109e34000001eb009e0078000040eb0002000700e8
:109e44000080fa00000006005600fa0040cf980097
:109e540071279800022f98001000200040079800f6
:109e64007e209000100798006a0f4700118380003d
:109e74001e007800ebf507001e00900010407800eb
:109e8400704798007e4090000004e00003003a0010
:109e94008080eb00212f9800b60137007e409000af
:109ea4000080fb00102f9800e00220009e28900004
:109eb400808f500005003200c00520009e289000cd
:109ec400808f5000b6003200030137001e0090005e
:109ed4000000e800100798001e0090001040780071
:109ee40070479800fe409000e0c2b30080cf50005d
:109ef40087003a001e0090000000e8001007980058
:109f04001e00900010407800704798001e007800f2
:109f14007011900080199000c0788000d178800082
:109f2400800f5100818f590003003a000080eb003c
:109f3400202f98008f0137001e00780080189000b1
:109f4400701090001e0178001019980021199800d3
:109f54001000200040079800e800470012c0b3003a
:109f64001e0078009dec0700200798002e0090004a
:109f74000000e00003003a008080eb00212f9800ed
:109f84007c0137002e009000b71007001e017800f6
:109f940070119800011998001e0078008018900034
:109fa400701090001e017800101998002119980073
:109fb4001e0078008018900070109000e00f500090
:109fc400e08f58001e003a001e007800c1c5b3009f
:109fd4004158980010c0b300604798000a00370049
:109fe4006e4090008080fb001e007800010040005d
:109ff400fc00400000c2b300804878006e4090002e
:10a004000040e800604798006e409000ea4f50001e
:10a01400f3ff3600c0788000d17880001e017800fc
:10a024001019980021199800c0788000d178800018
:10a034001e0178007011980001199800160037006d
:10a044009e007800e0c2b300c05898009e007800db
:10a05400e0c2b300d058980020c0b3006047980015
:10a064000a0037006e4090008080fb001e007800dc
:10a0740001004000fc00400000c2b30080487800aa
:10a084006e4090000040e800604798006e409000e9
:10a09400ea4f5000f3ff36000000eb004007980041
:10a0a400e800470012c0b3001e0078004bec070024
:10a0b4000000e00009003a000080eb00202f980027
:10a0c4002c0137001e0090000000e80010079800e3
:10a0d4001e0090001040780070479800fe409000e9
:10a0e400c0c5b30080cf5000f6ff32007e40900020
:10a0f4000004e00069ff3a00108380009e007800ad
:10a1040048f507008000eb00212f98001901370063
:10a114007e4090000004e00006003a0010838000b6
:10a124009e0078003ff507000000eb00202f980008
:10a1340010013700fe409000c0c5b30080cf50002e
:10a1440014003a00060037001e0090000000e800ea
:10a15400100798001e009000104078007047980087
:10a16400fe409000c0c5b30080cf5000f6ff32001f
:10a174007e4090000004e00048ff3a001083800015
:10a184009e00780027f507008000eb00212f98003f
:10a19400f80037000080eb00202f9800f50037000e
:10a1a4001e0090000000e800100798001e009000b8
:10a1b4001040780070479800fe409000c0c5b3007e
:10a1c40080cf500003003a008080eb00212f9800dc
:10a1d400e80037007e4090000004e00020003a00d0
:10a1e40012838000c0788000d178800070119800bc
:10a1f4000119980012838000c0788000d178800013
:10a20400101998002119980011838000c0c5b3006b
:10a21400c058980010c0b300604798000a00370087
:10a22400118380006e4090000080fb00008040009d
:10a23400fc00400000c2b300804878006e409000eb
:10a244000040e800604798006e409000ea4f5000dc
:10a25400f3ff36000000eb00202f9800c500370004
:10a26400c0788000d17880001e01780070119800b9
:10a2740001199800c0788000d17880001e01780010
:10a2840010199800211998009e007800c0c5b300e9
:10a29400c058980010c0b300604798000a00370007
:10a2a4006e4090008080fb001e007800010040009a
:10a2b400fc00400000c2b300804878006e4090006b
:10a2c4000040e800604798006e409000ea4f50005c
:10a2d400f3ff3600f1fe37000040eb0060479800c2
:10a2e4000f0037006e4090008080fb007e4190009c
:10a2f400c0fe200000804000024878006e409000bc
:10a304000040e800604798001e0090000000e8004c
:10a31400100798001e0090001040780070479800c5
:10a324007e4090000004e00007003200fe409000f0
:10a33400c0c5b30080cf5000030032006e409000cf
:10a34400ea4f5000e7ff36006e409000eb4f50009c
:10a3540018003a00060037001e0090000000e800d4
:10a36400100798001e009000104078007047980075
:10a374007e4090000004e0000e003200fe40900099
:10a38400c0c5b30080cf5000f3ff3a000900370086
:10a394006e4090008080fb00c0fe20008080400062
:10a3a40000c2b300804878006e4090000040e8008e
:10a3b400604798006e409000ea4f5000f4ff36006a
:10a3c4008040eb00c0fe2000da0707000040eb00ed
:10a3d400604798001a0037006e4090000081fb002f
:10a3e4006e4090000080fb009e0078007c004000de
:10a3f4000100400090407800000420000e0040005e
:10a4040000004100014878006e4090000081fb008c
:10a414006e4090008080fb00c0fe20000080400061
:10a42400904078001e007800020040007c0040004c
:10a43400014878006e4090000040e80060479800b2
:10a444006e409000ea4f5000e3ff36009e00780013
:10a4540020f6200073f407008041eb0012c0b30023
:10a464009e00780020f62000a6e307000000e0002c
:10a47400030032008080eb00212f98003d0037005c
:10a484000040eb00604798000f0037006e409000da
:10a494000081fb006e4090000080fb00fc00400047
:10a4a40020f6200000804000904078001e007800d4
:10a4b400020040007c004000014878006e4090009b
:10a4c4000040e800604798006e409000ea4f50005a
:10a4d400eeff3600207b8000317b80001e01780077
:10a4e40070119800011998001e00780080189000df
:10a4f400701090001e01780010199800211998001e
:10a504007e4090000004e00015003a0010838000b3
:10a514009e00780043f407000000eb00202f980011
:10a52400140037001e0090000000e8001007980097
:10a534001e00900010407800704798007e40900004
:10a544000004e00006003a00108380009e007800ba
:10a5540034f407008000eb00212f98000500370039
:10a56400fe409000c0c5b30080cf5000edff320024
:10a574004afe37002e2890000080fa0000000600f2
:10a584002200fa00500f9800610f98005e089000b6
:10a594000000e000030032006e089000006798009d
:10a5a40002003700a0c0b300006798008e609000de
:10a5b4006157980020f62000000f98000040eb003f
:10a5c400704f98000000eb00200798005e08900090
:10a5d4000000e00003003a0070ff2000200f980004
:10a5e400080037005e099000220f98006e08900062
:10a5f4000000e00003003a008001eb00730f9800b4
:10a604008e0137006e5090000000fb00800078003f
:10a614002e089000008040000000e900100f980010
:10a62400118380000e089000fef307000e089000ce
:10a63400c0589000e0c2b30080cf500097003a00a9
:10a644000e089000d0589000e0c2b30080cf5000b4
:10a6540092003a000e08900070119000801990004a
:10a66400520798006307980010002000400f9800dc
:10a674000e08900080189000701090000e09900051
:10a684001019980021199800f800470012c0b3006f
:10a694000e089000d1ea0700000f78001e00e000c9
:10a6a40003003a008001eb00730f98006301370048
:10a6b4001e007800ec0e07001079880021798800cc
:10a6c4001079800021798000e00f5000e08f58005d
:10a6d40006003a00c0788000d17880000e0990000e
:10a6e4007011980001199800050037001079800056
:10a6f400217980000e0990007011980001199800ca
:10a704000e08900080189000701090000e099000c0
:10a7140010199800211998000000eb00400f9800d0
:10a72400f800470012c0b3000e089000abea07001f
:10a73400000f78001e00e00003003a000000eb0068
:10a74400700f98003d0137001e007800c60e070008
:10a754001079880021798800110037004e08900094
:10a764000000e800400f9800f80047000041eb00ab
:10a774000e08900099ea0700000f78001e00e00020
:10a7840003003a008000eb00710f98002b013700a2
:10a794001e007800b40e0700107988002179880023
:10a7a40012798000237980005e009000ee00900012
:10a7b400800f5100818f5900e8ff3a001279800020
:10a7c400237980005e009000ee009000800f51001d
:10a7d400818f59000c003a001e0078001040780068
:10a7e400fb4f4000ddff32001e007800304890002f
:10a7f400e84f5000d9ff32001e0078003048900026
:10a80400ef4f5000d5ff32000000eb0030079800f6
:10a81400150037003e019000be0090001e00780035
:10a8240000804000904078000e0890000200400034
:10a834007c00400001487800138380003e019000b2
:10a84400be0090001e007800008040009040780018
:10a85400028041007c004000014878003e009000e6
:10a864000000e800300798003e009000ea0f500016
:10a87400e8ff34000e0890005e019000ee019000a5
:10a8840072109800031898000e0890005e01900062
:10a89400ee01900012189800231898000e089000fa
:10a8a400c0589000c0c5b30080cf500056003a0095
:10a8b400ae089000c0c5b300804878002e08900010
:10a8c4008000e8000040eb0080487800ae0990006a
:10a8d400730f9800d9003700a0c0b300604f9800f0
:10a8e400030037006e4890000040e900604f980074
:10a8f4006e4890000000fb008e0890007c00400031
:10a90400010040009040780000c2b30080cf5000a6
:10a91400f4ff32001a0037002e0090008000780007
:10a924002e089000008140006e4890000000fb005b
:10a934008e0890007c004000010040001040780028
:10a94400004978002e0090000000e80020079800dd
:10a954006e4890000040e900604f98006e509000ef
:10a964008000fb002e009000808f500004003a000d
:10a974000000eb002007980010c0b300704f98004f
:10a984006e4890000004e000e3ff3d002e009000bc
:10a99400800078002e08900080804000c0c5b3007d
:10a9a400804878002e0090000000e80020079800fe
:10a9b4006e5090008000fb002e009000808f5000ad
:10a9c40004003a000000eb002007980010c0b30018
:10a9d400704f98000e08900080189000701090003e
:10a9e4000e09900010199800211998000e08900083
:10a9f400950007000004e000030032000000eb00b3
:10aa0400700f98008d0037000e08900070119000b0
:10aa140080199000c0788000d1788000800f5100a8
:10aa2400818f5900acff3a002e0090000000e9002d
:10aa3400200798000000eb00300798007e48900043
:10aa44000004e00051003200ae009000410798007d
:10aa54001c0037003e009000800078002e08900013
:10aa64000080400010417800224798003e0090008a
:10aa7400800078002e089000008140002e00900095
:10aa8400800078002e08900000804000104078007c
:10aa9400004978002e009000800078002e08900075
:10aaa40000804000ae419000034878002e009000e2
:10aab4000000e900200798003e0090000000e80034
:10aac400300798002e009000be0090000100500056
:10aad4000000e000dfff3c004e0090000000e800b2
:10aae400300798009e0890002e08900000805000c7
:10aaf400200798001c0037003e009000800078007a
:10ab04002e08900000804000904078002147980073
:10ab14003e009000800078002e08900000814000e4
:10ab24002e009000800078002e08900000804000e5
:10ab340010407800004978002e00900080007800d2
:10ab44002e089000008040002e41900002487800ba
:10ab54002e0090000000e900200798003e009000bd
:10ab64000000e800300798002e009000be0090001e
:10ab7400010050000000e000dfff3c009e08900050
:10ab84000040eb00804878002a003700ae019000b6
:10ab9400430798001c0037003e00900080007800b6
:10aba4002e089000008040009040780021479800d3
:10abb4003e009000800078002e0890000081400044
:10abc4002e009000800078002e0890000080400045
:10abd40010407800004978002e0090008000780032
:10abe4002e089000008040002e419000024878001a
:10abf4002e0090000000e900200798003e0090001d
:10ac04000000e800300798002e009000be0090007d
:10ac1400010050000000e000dfff3c00ce00900087
:10ac24002e089000008040008000e8000040eb0007
:10ac340080487800ae099000730f98007e08900059
:10ac44000080fa00000006000e00fa005007980089
:10ac54001000200040079800e800470012c0b3002d
:10ac64005e0090005de90700000f78001e00e00020
:10ac740003003a00f00f200060079800b800370086
:10ac84001e007800780d070010798800217988006b
:10ac94001079800021798000e00f5000e08f580087
:10aca4001e003a005e009000c1c5b30041589800f0
:10acb4000040eb00704798000a0037007e40900087
:10acc4008080fb005e00900001004000fc0040001a
:10acd40000c2b300804878007e4090000040e80045
:10ace400704798007e409000ea4f5000f3ff360012
:10acf400c0788000d17880005e01900070119800c7
:10ad040001199800c0788000d17880005e0190001d
:10ad140010199800211998008f00370012798000cb
:10ad24002379800012079800230798001079800087
:10ad3400217980005e01900070119800011998003b
:10ad440010798000217980005e019000101998002c
:10ad540021199800e800470012c0b3005e0090007b
:10ad64001ee90700000f78001e00e00003003a000f
:10ad7400f30f200063079800790037001e00780065
:10ad8400390d070010798800217988001079800036
:10ad940021798000e00f5000e08f580006003a004f
:10ada400c0788000d17880005e0190007011980016
:10adb400011998000500370010798000217980007e
:10adc4005e01900070119800011998005e009000d7
:10add40080189000701090005e0190001019980087
:10ade400211998000000eb0040079800e800470094
:10adf40012c0b3005e009000f8e80700000f78006e
:10ae04001e00e00003003a00f00f200060079800e5
:10ae1400530037001e007800130d070010798800d6
:10ae24002179880011003700e80047000041eb0059
:10ae34005e009000e9e80700000f78001e00e000c3
:10ae440003003a00f10f2000610798004400370026
:10ae54004e0090000000e800400798001e007800b3
:10ae6400010d07001079880021798800127980008b
:10ae7400237980001e009000ae009000800f5100e6
:10ae8400818f5900e8ff3a0012798000237980000d
:10ae94001e009000ae009000800f5100818f590079
:10aea4000c003a001e00780010407800fb4f400070
:10aeb400ddff32001e00780030489000e84f50005b
:10aec400d9ff32001e00780030489000ef4f500048
:10aed400d5ff32001e0078001040780060479800cb
:10aee4000040eb00704798000e0037007e40900051
:10aef4000081fb007e4090008080fb001e007800f3
:10af040000804000904078005e0090000200400005
:10af14007c004000014878007e4090000040e8003a
:10af2400704798007e409000ea4f5000efff3600d3
:10af34005e0090001e019000ae0190007210980017
:10af4400031898005e0090001e019000ae0190006e
:10af540012189800231898008001eb0063079800ea
:10af64006e0090000080fa00000006000200fa0063
:10af7400000f78000001eb009e0078000000eb0059
:10af8400020007000080fa00000006001a00fa0020
:10af9400100f9800210f9800320f98002e0890008f
:10afa40010079800c0f22000000f780086180700f0
:10afb4000004e000030032000080eb00400f980022
:10afc4001b0137000040eb00504798000600370093
:10afd4001e0090000000e800100798005e409000fa
:10afe4000040e800504798001e0090001040780090
:10aff4000004e000050032001e009000904078003c
:10b00400c0c5b30080cf5000f1ff3a005e4090000d
:10b01400e84f5000060036000080eb00400f980017
:10b02400030137001e0090000000e800100798009c
:10b034001e00900090407800c0c5b30080cf50003f
:10b04400f8ff32001e009000104078000004e00079
:10b0540001003200dbff37002e0890001007980033
:10b06400118380001e0078006ef107000000370095
:10b074001e0090001040780050479800de40900079
:10b08400e0c2b30080cf50002b003a001e009000b5
:10b094000000e800100798001e009000104078009f
:10b0a40050479800de409000e0c2b30080cf5000cb
:10b0b40014003a00108380007011900080199000f1
:10b0c400c0788000d1788000800f5100818f5900b2
:10b0d40003003a000080eb00400f9800d4003700d2
:10b0e400b08d290050fb0700060037001e009000b9
:10b0f4000000e800100798001e009000104078003f
:10b1040050479800de409000c0c5b30080cf500087
:10b11400f6ff32005e4090000004e000d4ff3a00e5
:10b12400108380009e0078003ef107000080eb0051
:10b13400400f9800be003700de409000c0c5b30049
:10b1440080cf500036003a0012838000c07880001f
:10b15400d178800070119800011998001283800042
:10b16400c0788000d17880001019980021199800c7
:10b1740011838000c0c5b300c058980010c0b3004c
:10b18400504798000a003700118380005e40900009
:10b194000080fb0000804000fc00400000c2b300bf
:10b1a400804878005e4090000040e80050479800d6
:10b1b4005e409000ea4f5000f3ff36001e009000fe
:10b1c4000000e800100798001e009000104078006e
:10b1d40050479800de409000c0c5b30080cf5000b7
:10b1e40006003a00108380009e0078000df10700ed
:10b1f4000080eb00400f98008d0037005e40900007
:10b204000004e0009aff3a00108380009e0078005a
:10b2140004f107000080eb00400f98008400370021
:10b22400e60047000040eb00b048980000003700fb
:10b234001e00900010407800504798000040eb003a
:10b24400404798000f0037004e4090008080fb007c
:10b254005e4190006600470000804000024878008c
:10b264004e4090000040e800404798001e009000c7
:10b274000000e800100798001e00900010407800bd
:10b28400504798005e4090000004e0001100320036
:10b29400de409000c0c5b30080cf50000d003200e6
:10b2a4004e409000ea4f5000e7ff36000900370097
:10b2b4004e4090008080fb00660047008080400084
:10b2c40000c2b300804878004e4090000040e8007f
:10b2d400404798004e409000ea4f5000f4ff36007b
:10b2e4006600470090407800e0c2b30080cf500071
:10b2f40004003200660047008040eb000d040700a4
:10b304000c0037006600470090409000e0c2b30094
:10b3140080cf500004003a00e60047000040eb00f4
:10b32400a040980003003700e60047000040eb000f
:10b334009040980066004700bbfa07000000e00058
:10b3440014003a00060037001e0090000000e800d8
:10b35400100798001e009000104078005047980095
:10b36400de409000c0c5b30080cf5000f6ff32002d
:10b374005e4090000004e000adff3a0010838000be
:10b384009e007800a7f007000000eb00400f980033
:10b394002700370066004700280007000000e0008f
:10b3a40006003a00108380009e0078009df007009c
:10b3b4000080eb00400f98001d0037006600470036
:10b3c40099fa07000000e0000c00320010838000ae
:10b3d4009e00780093f007000080eb00400f980077
:10b3e400130037001e0090000000e80010079800ca
:10b3f4001e00900010407800504798001e009000f6
:10b4040090407800c0c5b30080cf5000f5ff3200f3
:10b414005e4090000004e00085ff3a001083800045
:10b424009e0078007ff007000000eb00400f9800ba
:10b434004e0890000080fa00000006001400fa0094
:10b44400000f980020f62000600798000000eb0031
:10b45400700798000040eb00004f78000b003700a5
:10b464001e81fb001e80fb00800078000e08900007
:10b4740000804000904078006e0090000200400080
:10b484007c004000014878001e4fe800a0c0b300d3
:10b494009e4f1000f2ff3600108380008018900049
:10b4a400701090006e0190007011980001199800be
:10b4b40010838000a0189000101890006e01900076
:10b4c40010199800211998006e0190006000b800ce
:10b4d40010019800210198006e0190006000b800ee
:10b4e400300198004101980010838000900078009a
:10b4f4006e00900001087800ee00470022c1b300fe
:10b504006e0090001ae807000000e000030032001b
:10b514000001eb00120f98004300370056d0bf0023
:10b524000004e0000c0032006e009000100078006f
:10b5340011c0b3006022b8006011b8000cf8070015
:10b54400e00f5000e08f5800030032008001eb0050
:10b55400130f9800340037006e00900070119000b3
:10b5640080199000c0788000d1788000800f51004d
:10b57400818f590004003a006000b8001007980059
:10b5840021079800050037006e00900070119000ac
:10b594008019900012079800230798006e0090000d
:10b5a40080189000701090006e019000101998009f
:10b5b40021199800ee00470012c0b3006e009000fd
:10b5c40006e70700500798005e0090000000e000c6
:10b5d40003003a008001eb00130f980012003700bb
:10b5e4005e009000200b0700300798004107980088
:10b5f4006e009000100078001e029000ae029000d1
:10b604003e019000ce0190000a0007000004e00013
:10b614000300320010002000100f980002003700d1
:10b624000001eb00120f98001e0890000080fa0041
:10b63400000006003e00fa005017980062179800b8
:10b6440073179800041f9800151f98006a0047009c
:10b65400200798000000eb00c08288000002200050
:10b66400300798005e10900010007800022020003f
:10b674008000eb00bddc0700ea004700e0c2b30035
:10b684008048780010002000400798000800370028
:10b69400ce0090006a0047008080400000c2b300e2
:10b6a400804878004e0090000000e80040079800b1
:10b6b4004e009000ea0f5000f5ff3600ea00470004
:10b6c40000c1b300b0489800ea0047000040eb0016
:10b6d400c0489800ee1090006a0047005108980096
:10b6e4006e109000fe10900002002000f3ff200076
:10b6f400000278008102780002007800830078005c
:10b7040000016200018062006102b800341f9800e9
:10b71400451f98003e189000ce189000c000dd0030
:10b7240000002000301f9800411f98003e18900030
:10b73400ce1890006112b800341f9800451f98007d
:10b744003e199000ce1990000200700083807000b2
:10b754004008de0001002000800078006a004700f5
:10b76400210898006a0147006000b8006009980049
:10b7740071099800ea00470020cbb300d048980034
:10b78400ea00470080272700f0009800ea004700fd
:10b79400002b230080089800ea0047000000eb001b
:10b7a40090089800ea0047000000eb00b0089800f9
:10b7b400ea0047000000eb00c00898000000eb001e
:10b7c400400798000c0037005e109000900078004d
:10b7d4004e00900000814000ae0090004e009000aa
:10b7e4000080400010407800004978004e0090002e
:10b7f4000000e80040079800ce0090003e00900052
:10b80400808f5000f0ff3900ea004700e0c2b30027
:10b81400904098008e1890006a00470051089800e4
:10b824000e1890009e18900002002000f3ff2000e4
:10b83400000278008102780002007800830078001a
:10b8440000016200018062006102b800541f980088
:10b85400651f98005e189000ee189000c000dd008f
:10b8640000002000501f9800611f98005e1890008f
:10b87400ee1890006112b800541f9800651f9800dc
:10b884005e199000ee199000020070008380700031
:10b894004008de0001002000800078006a004700b4
:10b8a400210898000000eb00400798000e003700c4
:10b8b4005e109000900078004e0090008080400060
:10b8c4003e00900000814000ae0090004e009000c9
:10b8d4000080400010407800004978004e0090003d
:10b8e4000000e80040079800ce0090003e00900061
:10b8f400808f5000eeff39006e119000fe11900011
:10b904005e10900001f00700008fbe005e109000f2
:10b91400100178008041eb001e00be00c315070033
:10b924000004e00003003a008001eb00231f9800ac
:10b934000200370014002000241f98002e189000e5
:10b944000080fa00000006000400fa00000f7800ee
:10b9540021479800ae4190000001eb009e00780062
:10b964000040eb00020007000080fa00000006001f
:10b974002200fa00005f9800510f9800620f9800af
:10b98400635f9800c0f220003007980020f6200082
:10b99400200798000000eb0040079800ec004700e7
:10b9a400e08d29000b000900b0587800c100b100f7
:10b9b400c000b100118380003e00900019ef070021
:10b9c4005e08900018f907000000e0000300320050
:10b9d4000080eb00001798000d02370010838000f0
:10b9e4007011900080199000c0788000d178800098
:10b9f400800f5100818f590006003a0010838000a7
:10ba0400be00900007ef07000080eb0000179800cd
:10ba1400ff0137004e0090000000e8004007980046
:10ba240010838000e800470012c0b300ebe5070074
:10ba3400100798001e0090000000e0001000320083
:10ba44001e009000080a0700407988005179880098
:10ba54004e0090000000e80040079800108380002a
:10ba6400e80047000041eb00dce507001007980000
:10ba74001e0090000000e000070032000c003700b8
:10ba840010838000be009000e6ee07000080eb000b
:10ba940000179800de01370010838000be0090007c
:10baa400e0ee07000080eb0000179800d801370093
:10bab4006e5890000004e00021003a001b0037009b
:10bac4001e00900010407800fb4f4000060032003a
:10bad40010838000be009000d2ee07000080eb00cf
:10bae40000179800ca0137004e0090000000e800db
:10baf4004007980010838000e80047000041eb00f5
:10bb0400b6e50700100798001e0090000000e00052
:10bb140006003a0010838000be009000c1ee0700ca
:10bb24000080eb0000179800b90137001e00900058
:10bb3400104078000004e000e1ff3a007201370091
:10bb44000040eb0027efb7000000eb00000f780087
:10bb54006a0137001e009000104078000004e000e5
:10bb6400b90032001e00900010407800fb4f4000e6
:10bb7400930032001e00900030489000e84f5000bf
:10bb84008f0032001e00900030489000ef4f5000ac
:10bb94008b0032001e009000304890000080fb00b3
:10bba4004400de00610060000004e0003c0032005c
:10bbb4001e0fe8006c004700000178006000b80028
:10bbc4000089be00640141006000b8000089be0025
:10bbd400640141006000b8000089be000040eb0031
:10bbe40026efb7000d00370026cfbf000081fb0011
:10bbf40026cfbf008080fb001e0090000080400024
:10bc0400904078006c004700000041000148780033
:10bc140026cfbf000040e80026efb70026cfbf00c4
:10bc2400ea4f5000f0ff36006c0047007ef8070032
:10bc34000000e0000600320010838000be00900087
:10bc440078ee07000080eb000017980070013700c1
:10bc54001083800070119000801990003e009000c5
:10bc64008018900070109000800f5100818f59004f
:10bc740006003a0010838000be00900069ee0700c1
:10bc84000080eb00001798006101370020002000bd
:10bc94004007980010c0b30060f0b7004b003700b5
:10bca4006c004700000178006000b8000089be0005
:10bcb400640141006000b8000089be0064014100d5
:10bcc4006000b8000089be000040eb0026efb7001a
:10bcd4000e00370026cfbf000081fb0026cfbf0037
:10bce4008080fb001e00900000804000904078009f
:10bcf4002e009000020040007c00400001487800c3
:10bd040026cfbf000040e80026efb70026cfbf00d3
:10bd1400ea4f5000efff3600ae009000e0fc200038
:10bd240080087800ce0090002e009000411098000a
:10bd34001083800080189000701090002e019000f5
:10bd4400701198000119980010838000a0189000c9
:10bd5400101890002e0190001019980021199800d5
:10bd64002e0190006000b800100198002101980095
:10bd74002e0190006000b800300198004101980045
:10bd8400e800470012c0b3002e009000e2e907006b
:10bd94000000e0000600320010838000be00900026
:10bda40020ee07000080eb00001798001801370010
:10bdb4004e0090000000e8004007980003003700a0
:10bdc4004e0090000000e8004007980060d0bf00db
:10bdd4000004e0000e0032000040eb0060f0b70009
:10bde40012838000108380008018900070109000ef
:10bdf400101998002119980010838000e80047006a
:10be040012c0b300f5e407001007980005003700de
:10be140010838000e80047000041eb00efe40700d6
:10be2400100798001e0090000000e000b3003a00e4
:10be340010838000be009000faed07000080eb0044
:10be440000179800f20037001e00e000a90032003d
:10be54000000eb00500798001283800010838000dc
:10be64008018900070109000101998002119980003
:10be740010838000ea00470012c0b300d7e4070033
:10be8400100798001e0090000000e00006003a0031
:10be940010838000be009000e2ed07000080eb00fc
:10bea40000179800da0037001e009000ee08070023
:10beb40050079800b08d2900dbf707000000e00070
:10bec4000600320010838000be009000d5ed07000c
:10bed4000080eb0000179800cd0037002000200000
:10bee400400798001283800010838000801890001f
:10bef4007010900010199800211998001083800088
:10bf0400e800470012c0b300b4e40700100798002b
:10bf14001e0090000000e00006003a00108380003c
:10bf2400be009000bfed07000080eb0000179800f2
:10bf3400b70037001e009000cb0807001079880076
:10bf440021798800150037004e0090000000e800b9
:10bf54004007980010838000e80047000041eb0090
:10bf64009ee40700100798001e0090000000e00007
:10bf740006003a0010838000be009000a9ed07007f
:10bf84000080eb0000179800a10037001e0090000d
:10bf9400b508070010798800217988005e009000b8
:10bfa4006101b8001079800021798000800f510070
:10bfb400818f5900e4ff3a005e0090006101b800ef
:10bfc4001079800021798000800f5100818f590001
:10bfd40008003a001e00900010407800fb4f40001b
:10bfe400d9ff32001e00900030489000e84f500006
:10bff400d5ff32006c004700000178006000b800f3
:10c004000089be00640141006000b8000089be00e0
:10c01400640141006000b8000089be000040eb00ec
:10c0240026efb7000d00370026cfbf000081fb00cc
:10c0340026cfbf008080fb001e00900000804000df
:10c04400904078006c0047000000410001487800ef
:10c0540026cfbf000040e80026efb70026cfbf0080
:10c06400ea4f5000f0ff36006c0047006b000700f9
:10c074000000e0000600320010838000be00900043
:10c0840068ed07000080eb0000179800600037009f
:10c094004e0090000000e8004007980012838000e2
:10c0a4001083800080189000701090001019980080
:10c0b4002119980010838000e800470012c0b300e3
:10c0c40046e40700100798001e0090000000e000fe
:10c0d40006003a0010838000be00900051ed070076
:10c0e4000080eb0000179800490037001e0fe9009c
:10c0f4000200370010c0b30027efb70027cfbf00fe
:10c104000004e00093fe32006c004700c1002000f0
:10c114001bf907000000e00006003a0010838000cd
:10c12400be0090003fed07000080eb000017980070
:10c13400370037006c004700000178006000b80049
:10c144000089be00640141006000b8000089be009f
:10c15400640141006000b8000089be000040eb00ab
:10c1640026efb7000e00370026cfbf000081fb008a
:10c174001183800026cfbf000080fb007c004000bc
:10c1840001004000904078006c004700000041002e
:10c194000148780026cfbf000040e80026efb70032
:10c1a40026cfbf00ea4f5000efff3600b08d2900c4
:10c1b4001df707000000e000060032001083800035
:10c1c400be00900017ed07000080eb0000179800f8
:10c1d4000f0037006c004700100007000000e0006b
:10c1e4000600320010838000be0090000ded0700b1
:10c1f4000080eb00001798000500370010838000d2
:10c20400be00900007ed07000000eb000017980047
:10c214000e1090000080fa00000006003e00fa00b4
:10c22400501f9800e81307000004e00003003200e8
:10c234000080eb00601f98003b00370011838000f2
:10c2440064004700f7ec07000040eb00004f780063
:10c254000b003700128380009e81fb001e80fb00d0
:10c26400800078005e1890000080400090407800c4
:10c27400030041007c004000014878001e4fe800a4
:10c28400a0c0b3009e4f1000f2ff3600118380005f
:10c2940020f62000e3ec0700108380008041eb00cf
:10c2a40012c0b30021f6200016dc07001007980026
:10c2b4001e0090000000e0000600320010838000a1
:10c2c400e4004700d7ec07000080eb00601f9800f3
:10c2d4001500370010838000810220008080400018
:10c2e4001083800012c0b3008be807001007980089
:10c2f4001e0090000000e00006003a001083800059
:10c30400e4004700c7ec07000000eb00601f980042
:10c314000500370010838000e4004700c1ec0700eb
:10c324000080eb00601f98006e1890000080fa00f7
:10c33400000006001000fa0060079800614f9800a2
:10c344000040eb0026efb7000d00370026cfbf00fa
:10c354000081fb0026cfbf000080fb008000780036
:10c364006e00900000804000904078000e00410074
:10c374000148780026cfbf000040e80026efb70050
:10c3840026cfbf00e74f5000f0ff360000c2b300d5
:10c39400004f980000c2b300104f980000c2b300d1
:10c3a400204f98000040eb00304f98009e407800ea
:10c3b40000c2b30080cf500002003a00f0c5b300c1
:10c3c400004f78006e49900011c0b3000e00780051
:10c3d40070f007000040eb0026efb7000d003700b7
:10c3e40026cfbf000080fb00800078006e00900024
:10c3f4008080400026cfbf000080fb000e0040007c
:10c40400104078008048780026cfbf000040e80044
:10c4140026efb70026cfbf00ea4f5000f0ff3600ea
:10c424000080fa00000006004800fa000027980087
:10c4340011279800222798006800470030079800c9
:10c444003e009000fc00400012c0b3000e2090009b
:10c45400cdef07000004e00003003a000080eb0089
:10c4640030279800410137002e2090008040eb00d7
:10c47400016898000040eb0026efb7000f0037007a
:10c4840026cfbf000081fb0026cfbf000080fb0049
:10c49400800078000e2090000080400090407800da
:10c4a4002e209000020040007800400001487800ef
:10c4b40026cfbf000040e80026efb70026cfbf001c
:10c4c400eb4f500008003e0026cfbf000080fb0069
:10c4d400800078000e20900000804000104078001a
:10c4e4000004e000e6ff3a0026cfbf008080fb0096
:10c4f4002e20900001004000f80040000040eb00b6
:10c50400804878001e209000804078002e20900003
:10c514005160980010838000801890007010900083
:10c52400800078002e20900031109800be0090000a
:10c53400e0fc2000800878003e0190006000b80014
:10c5440010019800210198003e0190006000b8009d
:10c554003001980041019800be0090000000eb00fb
:10c56400c01098003e0090009e209000611098003a
:10c574001083800080189000701090003e0190009d
:10c58400701198000119980010838000a018900081
:10c59400101890003e01900010199800211998007d
:10c5a400be00900020f620001eec070013c0b3006c
:10c5b40012c0b30021f620003e00900051db0700ba
:10c5c400200798002e0090000000e00003003200d5
:10c5d4000080eb0030279800e40037003e00900014
:10c5e40040109000701f9800e10320008e804000ee
:10c5f40022c7b3003e00900031dc070020079800fa
:10c604002e0090000000e000d6003a003e009000aa
:10c6140060109000e80f5000650032003e0090006a
:10c6240060109000f00f5000610032000040eb00f9
:10c6340026efb7000040eb002047980011003700b8
:10c6440026cfbf000081fb002e4090000080fb003d
:10c65400be0090007c004000010040009040780043
:10c664002e209000000041000148780026cfbf0032
:10c674000040e80026efb7002e4090000040e8009c
:10c68400204798002e409000e74f500009003e00dc
:10c694002e4090000080fb00be0090007c00400013
:10c6a400010040009040780000c2b30080cf5000e9
:10c6b400e3ff3a003e009000c060900000c2b30067
:10c6c40080cf50000a003a003e009000d0609000f5
:10c6d40000c2b30080cf500005003a003e00900035
:10c6e400e060900000c2b30080cf50000900320027
:10c6f40062f22000124178008280fb002e2090001c
:10c7040080804000e0c2b300804878000240e80026
:10c7140026efb70080c0b30020479800110037000f
:10c7240026cfbf000081fb002e4090000080fb005c
:10c73400be0090007c004000010040009040780062
:10c744002e209000000041000148780026cfbf0051
:10c754000040e80026efb7002e4090000040e800bb
:10c76400204798002e409000ea4f500009003e00f8
:10c774002e4090000080fb00be0090007c00400032
:10c78400010040009040780000c2b30080cf500008
:10c79400e3ff3a0026cfbf008080fb002e209000ec
:10c7a400808040000040eb00804878002f00370074
:10c7b4000040eb0026efb7000e00370026cfbf0085
:10c7c4000081fb0026cfbf000080fb00be0090006c
:10c7d4007c00400001004000904078002e20900032
:10c7e400000041000148780026cfbf000040e80067
:10c7f40026efb70026cfbf00ea4f5000efff360008
:10c8040026cfbf008080fb002e2090008080400057
:10c814000040eb008048780026cfbf000040e900cc
:10c8240026efb7000900370062f2200012417800b9
:10c834008280fb002e209000808040000040eb00ae
:10c84400804878000240e90026efb70026cfbf00f9
:10c854008080fb002e2090000080400090407800f3
:10c8640000c2b30080cf5000efff32003e009000c2
:10c8740060109000804078002e209000514898006d
:10c884003e009000a0089000100890002e21900017
:10c8940070019800010998003e009000601090001b
:10c8a4004400de000000a200610060000004e0001b
:10c8b4000e0032003e00900050089000010020005d
:10c8c400c001dd00020020003e00900040089000fe
:10c8d4000100200002004000838048002e219000c7
:10c8e4001009980021099800140037003e009000b8
:10c8f40081022000808040000041eb003e00900057
:10c9040036e20700000f78001e007800000890004f
:10c9140001002000c001dd00020020001e0078009c
:10c924007000900001002000020040008380480055
:10c934002e21900010099800210998003e009000d3
:10c94400c01090002e20900031089800ae20900076
:10c9540010c0b300806898008000eb003127980075
:10c96400020037000080eb00302798003e20900042
:10c974000080fa00000006004200fa00701f9800d0
:10c9840068004700300798007e1890000068900007
:10c994000004e00003003a000080eb000027980048
:10c9a400190137007e189000301090006101b80022
:10c9b400108380008018900070109000800f510048
:10c9c400818f5900030032000080eb00002798009b
:10c9d4000d0137003e009000fc0040007e189000de
:10c9e4007800400012c0b30067ee07000004e000c6
:10c9f40003003a000080eb00002798000201370092
:10ca0400be009000e0fc2000800878003e01900009
:10ca14006000b80010019800210198003e019000c8
:10ca24006000b80030019800410198007e18900021
:10ca3400300890008000e8003e009000411098000b
:10ca44007e189000506090008080fb003e009000b3
:10ca5400611098001083800080189000701090007e
:10ca64003e01900070119800011998001083800015
:10ca7400a0189000101890003e0190001019980022
:10ca840021199800be00900020f62000e5ea070076
:10ca940013c0b30012c0b30021f620003e00900082
:10caa40018da0700200798002e0090000000e0002c
:10cab400030032000080eb0000279800d20037000a
:10cac4003e00900060109000e80f500065003200b6
:10cad4003e00900060109000f00f500061003200a2
:10cae4000040eb00304798000040eb0020479800de
:10caf400110037003e4090000081fb002e40900062
:10cb04000080fb00be0090007c004000010040005b
:10cb1400904078007e1890000000410001487800a1
:10cb24003e4090000040e800304798002e409000be
:10cb34000040e800204798002e409000e74f500046
:10cb440009003e002e4090000080fb00be009000d3
:10cb54007c004000010040009040780000c2b30017
:10cb640080cf5000e3ff3a003e009000c060900088
:10cb740000c2b30080cf50000a003a003e0090008b
:10cb8400d060900000c2b30080cf500005003a008e
:10cb94003e009000e060900000c2b30080cf5000df
:10cba400090032003e4090008080fb007e18900017
:10cbb40080804000e0c2b300804878003e4090008e
:10cbc4000040e8003047980080c0b3002047980038
:10cbd400110037003e4090000081fb002e40900081
:10cbe4000080fb00be0090007c004000010040007b
:10cbf400904078007e1890000000410001487800c1
:10cc04003e4090000040e800304798002e409000dd
:10cc14000040e800204798002e409000ea4f500062
:10cc240009003e002e4090000080fb00be009000f2
:10cc34007c004000010040009040780000c2b30036
:10cc440080cf5000e3ff3a003e4090008080fb001c
:10cc54007e189000808040000040eb0080487800ff
:10cc64002f0037000040eb00304798000e003700db
:10cc74003e4090000081fb003e4090000080fb009d
:10cc8400be0090007c00400001004000904078000d
:10cc94007e18900000004100014878003e4090005a
:10cca4000040e800304798003e409000ea4f5000b2
:10ccb400efff36003e4090008080fb007e1890001d
:10ccc400808040000040eb00804878003e409000a7
:10ccd4000040e90030479800090037003e409000ca
:10cce4008080fb007e189000808040000040eb00b4
:10ccf400804878003e4090000040e90030479800aa
:10cd04003e4090008080fb007e1890000080400030
:10cd14009040780000c2b30080cf5000efff320093
:10cd24003e00900060109000804078007e189000d3
:10cd3400514898003e009000a00890001008900010
:10cd44007e19900070019800010998003e0090003f
:10cd5400601090004400de000000a200610060004a
:10cd64000004e0000e0032003e00900050089000e5
:10cd740001002000c001dd00020020003e00900000
:10cd84004008900001002000020040008380480019
:10cd94007e199000100998002109980014003700aa
:10cda4003e00900081022000808040000041eb00a2
:10cdb4003e00900009e10700000f78001e00780093
:10cdc4000008900001002000c001dd0002002000e6
:10cdd4001e00780070009000010020000200400056
:10cde400838048007e19900010099800210998005a
:10cdf4003e009000c01090007e189000310898000a
:10ce04000000eb00002798000e2090000080fa003c
:10ce1400000006000600fa0020079800680057008a
:10ce2400100798001e019000ceb897002e009000c5
:10ce340004000700000f78001e0078000080fa004c
:10ce4400000006007000fa00702f98000137980067
:10ce5400123798000000eb00500f98000e3090003d
:10ce640010407800405f9800cd043700ce58900001
:10ce740050c2b30080cf5000b8043a000040eb0029
:10ce8400105f98000040eb00005f98000040eb004a
:10ce9400705798000040eb00605798000040eb008a
:10cea400505798000040eb00405798000e30900017
:10ceb4000000e800003798000e3090001040780021
:10cec400405f9800360037004e5890000080fb0009
:10ced40050379800b0022000de309000808f500060
:10cee4001a003200b00220005e319000800f510021
:10cef40009003c0000022000de319000808f5100c8
:10cf040016003200300220005e329000800f520082
:10cf1400160032001c003700d0022000de329000e0
:10cf2400808f520005003200000320005e33900021
:10cf3400800f530011003200130037001e58900078
:10cf44000004a000105f98000f0037001e589000e6
:10cf54000014a000105f98000b0037001e589000ca
:10cf64000024a000105f9800070037001e589000ae
:10cf74000034a000105f9800030037001e58900092
:10cf84000044a000105f98000e3090000000e800fc
:10cf9400003798000e30900010407800405f9800f1
:10cfa400ce589000d0c2b30080cf5000c6ff3200ec
:10cfb400ce589000b0c2b30080cf5000c2ff320000
:10cfc400ce58900000c2b30080cf5000beff3200a4
:10cfd400ce58900030c2b30080cf5000baff320068
:10cfe400ce58900000c3b30080cf5000b6ff32008b
:10cff400ce589000a0c2b30080cf500019003a0070
:10d004001e3090000080e900103798001e30900018
:10d0140090037800370798003e0090000000e0007d
:10d0240007003d001e5890000004a000105f980007
:10d034003e0090000040ea00005f980002003700c4
:10d044003e009000005f98000e3090000000e80061
:10d05400003798000e30900010407800405f980030
:10d064001a0037000040eb00205798000f003700eb
:10d074002e5090000080fb006a00b90080407800c8
:10d084004e58900080c0400000cdb30000c0400066
:10d09400205798000e3090000000e80000379800f8
:10d0a4000e30900010407800405f98004e58900079
:10d0b4008080fb0000fd2f0000804000e90f50003d
:10d0c400ebff36002e509000005f98001e58900031
:10d0d4000080fb00610060000004e00004003200f6
:10d0e4001e589000f1ceb30001406000105f98001c
:10d0f400ce589000e0c2b30080cf50003a003a000e
:10d104000e3090000000e800003798000e309000c8
:10d1140010407800405f9800ce589000a0c2b30041
:10d1240080cf500014003a001e3090000080e900c7
:10d13400103798001e309000900078003107980056
:10d144003e0090000000e000040035003e00900026
:10d154007057980010c0b300605798000e309000cc
:10d164000000e800003798000e309000104078006e
:10d17400405f98001c0037000040eb0020579800e7
:10d184000f0037002e5090000080fb006a00b900a9
:10d19400804078004e58900080c0400000cdb3001d
:10d1a40000c04000205798000e3090000000e800b6
:10d1b400003798000e30900010407800405f9800cf
:10d1c4004e5890008080fb0000fd2f00008040003e
:10d1d400e90f5000ebff36002e5190007257980073
:10d1e40010c0b30060579800ce58900080c6b300ba
:10d1f40080cf500013003a000e3090000000e80089
:10d20400003798000e30900010407800405f98007e
:10d21400ce58900080c6b30080cf500035003a004d
:10d2240030c0b300505798000e3090000000e80062
:10d23400003798000e30900010407800405f98004e
:10d244002c003700ce58900040c7b30080cf500068
:10d2540004003200ce589000a0c7b30080cf500025
:10d2640007003a000e3090000000e80000379800f4
:10d274000e30900010407800405f98001d00370089
:10d28400ce58900010c7b30080cf50000400320085
:10d29400ce589000a0c6b30080cf500009003a00d9
:10d2a40010c0b300505798000e3090000000e80002
:10d2b400003798000e30900010407800405f9800ce
:10d2c4000c003700ce589000c0c6b30080cf500089
:10d2d40008003a0020c0b300505798000e30900068
:10d2e4000000e800003798000e30900010407800ed
:10d2f400405f98004e5890000080fb006102b90026
:10d3040064379800753798008007200001002000da
:10d314006e339000fe339000800f5300818f5b00ca
:10d3240099033e006e309000fe30900000600100d2
:10d3340078003700940337009303370092033700d3
:10d3440091033700900337008f0337008e033700b3
:10d354008d0337008c0337008b0337008a033700b3
:10d3640089033700880337008703370086033700b3
:10d3740085033700840337008303370082033700b3
:10d3840081033700800337007f0337007e033700b3
:10d394007d0337007c0337007b0337007a033700b3
:10d3a40079033700780337007703370076033700b3
:10d3b40075033700740337007303370072033700b3
:10d3c40071033700560037006f0337006e033700d0
:10d3d4006d0337006c0337006b0337006a033700b3
:10d3e40069033700680337006703370066033700b3
:10d3f40065033700640337006303370062033700b3
:10d4040061033700600337005f0337005e033700b2
:10d414005d0337005c0337005b0337005a033700b2
:10d4240059033700580337005703370056033700b2
:10d434005503370054033700eb003700520337001d
:10d4440051033700500337004f0337004e033700b2
:10d454004d0337004c0337004b0337004a033700b2
:10d4640049033700480337004703370046033700b2
:10d474003901370044033700430337006e00370097
:10d4840041033700400337003f0337003e033700b2
:10d49400d50037003c0337003b0337003a0337001d
:10d4a40039033700380337003703370036033700b2
:10d4b4003503370034033700cb003700240037002e
:10d4c400c5003700300337002f0337002e03370021
:10d4d4002d033700c00037002b0337002a03370021
:10d4e4002903370028033700ea023700be0037005b
:10d4f4001901370024033700230337004e00370097
:10d5040021033700b80037001f0337001e0337001c
:10d51400b50037000e3090000000e9000037980095
:10d52400fe28900050c2b30025030700e10f40001d
:10d5340003003a008080eb00413798001d03370058
:10d544005e0890000000e800500f98000e033700ba
:10d554000040eb00305798000e589000e14f500007
:10d56400080036000e5890000040e900305798003b
:10d574003e5090008080fb005e0890000100400057
:10d58400500f98003e5090000004e000100032005c
:10d594001e5890000080fb00610060000000e00065
:10d5a4000b003a0002c2b300be5090007e289000e7
:10d5b400150307000004e000030032000081eb00c3
:10d5c40042379800fb0237000040eb0030579800c8
:10d5d4001e3090000080e900103798001e30900043
:10d5e40010007800405f98004e589000fe2890008c
:10d5f400f3020700e10f400003003a008081eb00d2
:10d6040043379800eb0237005e0890000000e80002
:10d61400500f980002c2b300be5090007e289000c4
:10d62400f90207000004e000d70232000082eb0098
:10d6340044379800df0237001e3090000080e90074
:10d64400103798001e30900090027800450798002b
:10d654004e009000e6d40700300798006e5090000a
:10d664000004e000080032003e0090008040780092
:10d674007e50900080cf5000030036007e50900012
:10d684000080fb00300798003e0090008040780046
:10d694000e58900080cf5000020036003e009000eb
:10d6a400005f98003e009000804078000e58900083
:10d6b40001405000305798003e5090008080fb009d
:10d6c4005e08900001004000500f98006e509000da
:10d6d4000004e00006003200fe5090000e58900056
:10d6e40080cf5000020031007e539000065f980006
:10d6f4001e5890000080fb00610060000000e00004
:10d704000b003a0002c2b300be5090007e28900085
:10d71400bd0207000004e000030032008083eb0038
:10d7240047379800a30237000040eb0030579800b9
:10d734000040eb00205798004e0090001040780005
:10d74400405f9800140037004e589000fe28900067
:10d754009b020700e10f400003003a000080eb0049
:10d7640040379800930237005e0890000000e800fc
:10d77400500f98002e5090000040e8002057980069
:10d784004e0090000000e800400798004e00900012
:10d7940010407800405f98004e5890000004e0006c
:10d7a40004003200ae5090000e58900080cf50001c
:10d7b400e5ff390002c2b300be5090007e289000fd
:10d7c400910207000004e0006f0232008080eb0049
:10d7d40041379800770237001e58900001c8b30003
:10d7e40001407000105f98005e509000e24f5000be
:10d7f4001b003a001e5890000004e0000c003d009d
:10d804001e30900064005000103798001e309000c5
:10d814001000be0050079800610798004f88de0092
:10d82400cf80de0070079800000f98006600370074
:10d834001e30900064005000103798001e30900095
:10d844001000be0050079800610798000000eb002c
:10d85400700798000000eb00000f98005a00370092
:10d864005e509000e34f50001f003a001e58900095
:10d874000004e0000e003d001e3090000080e9002e
:10d88400103798001e309000100078000000fb0054
:10d89400cf80de00010178008201780050079800f3
:10d8a4006107980072079800030f9800460037003c
:10d8b4001e3090000080e900103798001e30900060
:10d8c400100078000080fb0001002000020020000e
:10d8d4000300200050079800610798007207980021
:10d8e400030f9800380037005e509000e14f50005d
:10d8f40019003a001e5890000004e0000b003d009f
:10d904001e30900068005000103798001e309000c0
:10d914005001be004000be00500798006107980007
:10d9240072079800030f9800270037001e309000fc
:10d9340068005000103798001e3090003002be007e
:10d944002003be00540798006507980076079800e6
:10d95400070f98001c0037001e5890000004e000d8
:10d964000d003d001e3090000080e9001037980043
:10d974001e30900010007800cf80de000101780096
:10d984008201780050079800610798007207980098
:10d99400030f98000c0037001e3090000080e9004f
:10d9a400103798001e30900010007800010020000d
:10d9b400020020000300200050079800610798002f
:10d9c40072079800030f98006e5090000004e00066
:10d9d40002003a0010c0b300705798000040eb00fa
:10d9e400404798000040eb00304798007d00470016
:10d9f400f5032000050f4000fd0047000040eb0048
:10da040080c098000040eb0030579800a0c0b300dd
:10da1400505798004e5890000080fb003037980013
:10da2400200620003e339000800f53001e00320079
:10da340020062000be339000808f53000d003c0070
:10da440000052000be309000808f5000200032007e
:10da5400800520003e319000800f51001f003200ed
:10da640020042000be319000808f51000e0032004f
:10da74001e003700000720003e329000800f520045
:10da84001300320080072000be329000808f5200c5
:10da940012003200f00620003e339000800f530045
:10daa400060032001100370020c0b3005057980020
:10dab40010c0b300405798000c00370080c0b3007a
:10dac4005057980030c0b300405798000700370003
:10dad4004e58900068404000405f980000c1b30079
:10dae4005057980040c0b300405798001e5890000b
:10daf4000004e000040035001e58900091cfb300ec
:10db040001406000105f98001e5890000004e0007f
:10db14001d003d005e009000ee0090007e0190002c
:10db24008e099000e00f5000e08f5800e00f59007c
:10db3400e08f590014003d005e029000ee02900058
:10db44007e0390008e0b90006000b8006011b80056
:10db5400040050008580580006015900878159004f
:10db6400500798006107980072079800030f980007
:10db7400d0c2b300204798004e4090000040e80017
:10db8400404798001a0037001e5890000080fb00a0
:10db94000000d100610060000004e00006003200d3
:10dba400b0c2b300204798004e4090000040e80007
:10dbb400404798000e0037001e5890000080fb007c
:10dbc4004200de00610060000004e0000600320054
:10dbd40000c2b300204798004e4090000040e80087
:10dbe40040479800020037000040eb0020479800af
:10dbf4007e5090000004e00009003a005e009000ae
:10dc0400ee0090007e0190008e099000e00f50001d
:10dc1400e08f5800e00f5900e08f59008100320076
:10dc24004e5090000004e0000b003200de00900033
:10dc34005e5090000081fb00110009008280d80032
:10dc44008000fd0080007800a08c290061407800ed
:10dc5400205798000e0037005e5090000082fb00b1
:10dc64000500200006002000070020005e00900050
:10dc7400ee0090007e0190008e09900005d407000c
:10dc8400a48c29000000420010407800205798001e
:10dc9400ce58900080c5b30080cf500008003a00f1
:10dca400ae50900000c6b30080cf50000400360090
:10dcb4002e50900001ceb300014040002057980040
:10dcc4004e5090000004e000130032004e509000cb
:10dcd4000082fb005e009000ee0090007e01900048
:10dce4008e099000840378008703e900050033005f
:10dcf4008301d1000281d3008180d3000080d3004e
:10dd0400f9ff3700500798006107980072079800e0
:10dd1400030f98000e0037005e5090000082fb0055
:10dd24000500200006002000070020005e0090008f
:10dd3400ee0090007e0190008e099000ced3070083
:10dd4400500798006107980072079800030f980025
:10dd5400ae5090001e007800014878001e0fe900c4
:10dd64004e4090000040e800404798005e0090005c
:10dd7400ee0090007e0190008e099000e00f5000ac
:10dd8400e08f5800e00f5900e08f5900a4ff3a00db
:10dd94001e5890000080fb004300de00610060001c
:10dda4000004e00021003200ce589000f0c6b30019
:10ddb40080cf500008003a00fe5090004e40900082
:10ddc40080cf500019003e004e4090000040e80013
:10ddd4007057980015003700ce58900080c7b300e4
:10dde40080cf50000c003200ce58900080c5b300a4
:10ddf40080cf500008003200ce58900020c6b300f7
:10de040080cf500004003200ce58900020c4b300ec
:10de140080cf500005003a0020c0b300304798007e
:10de2400020037000040eb00404798001e58900065
:10de34000080fb004400de00610060000004e0009c
:10de4400090032008e5890007e50900080cf500020
:10de5400050036006e5090000004e00002003a0015
:10de64000e58900070579800fe5090004e4090005d
:10de740080cf5000050036007e509000ce409000c8
:10de84000140500070579800020037000040eb003a
:10de9400705798000e5890000081fb007e5090004f
:10dea4008080fb004e4090000080fb00808040009a
:10deb4003e4090000080fb0000804000800f510035
:10dec400090034008e5890007e50900000c050002d
:10ded400804078004e40900080c050003e4090004a
:10dee40000c05000305798001e5890000080fb007e
:10def400610060000000e00013003a003e50900012
:10df04000004e0001000320002c2b300be509000d2
:10df14007e289000bc0007000004e00003003200eb
:10df24008080eb0041379800a20037003e509000fb
:10df34008080fb005e08900001004000500f9800b4
:10df44000040eb00305798002e4090000004e000a1
:10df5400080032002e409000fe2890009800070030
:10df6400e10f400003003a000081eb0042379800c3
:10df7400900037003e4090000004e00010003200a2
:10df8400fe28900000c3b3008d000700e10f40009d
:10df940003003a008081eb00433798008500370086
:10dfa4004e589000fe28900085000700e10f4000c5
:10dfb40003003a000082eb00443798007d003700ec
:10dfc40002c3b300fe5090007e2890008e0007002c
:10dfd4000004e000030032008082eb004537980023
:10dfe400740037001e0fe8001e007800104078000f
:10dff400205798000c0037002e509000fe28900007
:10e004006f000700e10f400003003a000083eb00bb
:10e0140046379800670037001e0fe8001e0078009e
:10e0240010407800205798002e5090000004e00023
:10e03400f1ff3a0002c2b300be5090007e28900067
:10e04400710007000004e000030032008083eb004d
:10e0540047379800570037007e5090008080fb00bf
:10e064004e4090000080fb00808040003e509000b5
:10e074000080fb00808040003e4090000080fb0058
:10e08400808040005e08900001004000500f98001e
:10e094003d0037005e5090000080fb002037980060
:10e0a4002e309000e20f500007003200ae30900096
:10e0b400e38f5000190032002e319000e10f51001f
:10e0c4000a0032001d0037001e3090000080e90075
:10e0d400103798001e309000100178005e08900000
:10e0e400cf80de000089be00270037001e3090007c
:10e0f4000080e900103798001e309000100278006c
:10e104005e089000cf80de00010178008201780073
:10e11400009abe000292be001b0037001e30900021
:10e124000080e900103798001e30900090007800bd
:10e134005e08900080487800130037001e3090007d
:10e144000080e900103798001e309000100078001d
:10e15400de099000030878000b0037004e58900049
:10e16400fe28900016000700e10f400003003a006b
:10e174000082eb00443798000e0037005e089000e0
:10e184000000e800500f98000e3090000000e800f6
:10e19400003798000e30900010407800405f9800df
:10e1a4004e5890000004e00030fb3a00de0a900074
:10e1b400453798004e3090000080fa0000000600b9
:10e1c4000600fa00004f7800110798009e019000a5
:10e1d40012002000110020000e0078001fe6070046
:10e1e400e10f5000030032000080eb00200798008c
:10e1f400020037000000eb00200798002e0090007a
:10e204000080fa00000006000600fa00000f780003
:10e214002147980032479800080037009e00780094
:10e224003e409000e6ff0700e10f400003003a0083
:10e234001000200020079800080037002e409000ae
:10e244000040e900204798002e409000e14f400034
:10e25400f2ff3a000000eb00200798002e00900027
:10e264000080fa00000006000600fa00200798006b
:10e274006000b800008fbe002e00900020089000bf
:10e2840001002000008fbe001e00be00c000dd00a3
:10e2940000002000008fbe002e0090005008900067
:10e2a400010020001e1f70001e9770001e00be009b
:10e2b4000080fa00000006000400fa00000f780055
:10e2c400110798001e0090001e00400010407800c6
:10e2d4000080fb000080fa00000006000800fa003d
:10e2e4002007980031079800be0090002e0090008f
:10e2f400008040009040780031479800be009000b4
:10e304002e009000008040000000e800904078005b
:10e31400214798002e4090000080fb00000f7800f9
:10e324001e0078004800dd00000f78003e40900099
:10e334000080fb001e0f70001e0078000080fa00b1
:10e34400000006000c00fa004007980051079800ee
:10e35400de0090004e009000e0ff070030079800b8
:10e364005e0090008080e8004e009000dbff070014
:10e37400200798002e00900001002000008fbe00ae
:10e384001e00be00c000dd0000002000008fbe00a3
:10e394003e009000010020001e1f70001e977000b8
:10e3a4001e00be000080fa00000006000200fa0011
:10e3b400f00f200070248800f00f20005024880003
:10e3c400f009200080248800b00f20006024880019
:10e3d4008804a800002021004800de00c024880032
:10e3e4009424a8009424a9000000eb00b024880021
:10e3f4000040eb00004f7800070037001e80fb0050
:10e40400c200dd0000202100008140006000b8004f
:10e414000089be001e4fe80030c0b3009e4f1000bc
:10e42400f6ff3600d0002000502588000300370096
:10e43400a048200031c0b300a70407008ac4bf006d
:10e44400684060000004e000f9ff3a000040eb007f
:10e4540014e8b700818120000040eb00a040980040
:10e4640094a4a90040202100004188000040eb0052
:10e4740011e8b7000040eb0010e8b7000080fa0094
:10e48400000006000200fa0010c8bf000004e0000b
:10e4940010003a000000eb00a02488000000eb000c
:10e4a40060248800010037009404a80094c4bf00cd
:10e4b400614060000004e000fbff320010c0b300c4
:10e4c40010e8b7000000eb003025880000012000b0
:10e4d4004025880010c8bf00e14f500008003a00f2
:10e4e400f00f2000502488000000eb006024880016
:10e4f4008c04a8008c84a80020c0b30010e8b700e6
:10e5040080c4bf00704060000004e00005003200d9
:10e5140082c4bf00704060000004e00001003200cb
:10e524008200070088c4bf00624060000004e0006d
:10e534005c003a008ac4bf00614060000004e0004f
:10e54400150032008cc4bf00614060000004e0008c
:10e554001100320095ff070040c0b30010e8b70077
:10e56400008020001090880080c0b30000f2b70043
:10e57400112021009140780030c0b30000c0600039
:10e5840001f2b7001120210091407800c0c8b30007
:10e5940000c0700001f2b7008ac4bf007040600080
:10e5a4000004e000050032008cc4bf00704060002d
:10e5b4000004e00001003200540007008ac4bf00d8
:10e5c400644060000004e000080032008cc4bf0016
:10e5d400644060000004e00004003200120c0700f4
:10e5e400a048200021c0b3003b0407008ac4bf0038
:10e5f40001c8b300014060000004e00006003200de
:10e604008cc4bf0001c8b300014060000004e000f6
:10e6140001003200250007008ac4bf006240600088
:10e624000004e000070032008cc4bf0062406000b8
:10e634000004e00003003200fe0b0700f00f20008e
:10e644007024880010c8bf00e34f50001500360046
:10e654008cc4bf00684060000004e0001100320078
:10e664000040eb00004f78000b0037008ac4bf0065
:10e67400684060000004e0000a003200902480003a
:10e6840062eab700a048200031c0b30012040700ba
:10e694002e0007001e4fe80030c0b3009e4f10004c
:10e6a400f2ff36000080fa00000006000000fa00c5
:10e6b400aac4bf00624060000004e0000e00320003
:10e6c400a05280009040900000c8b30080cf50005a
:10e6d40008003a00004180009040900040c8b30018
:10e6e40080cf500003003a00a1528000c0c8b3009c
:10e6f40090409800aa24a900a048200021c0b3009b
:10e70400f50307000080fa00000006000000fa008c
:10e714008284a800a048200041c0b300ee03070093
:10e72400bb0b07000080fa00000006000000fa009e
:10e73400ba0b07008284a9000048200041c0b3003e
:10e74400e50307000080fa00000006000000fa005c
:10e7540062cabf008080fb00b0ff2f000080600011
:10e764000000e0001b003a0062cabf008080fb008a
:10e77400c00f2000008060004280de004200dd0007
:10e78400800078000020210000804000a052880012
:10e79400a0528000b052880061a5200060a520002e
:10e7a4001040780080487800a0528000104090000b
:10e7b400c2c3b3008240600040c3b30080cf5000a6
:10e7c40002003a000c00070009003700210007008e
:10e7d4000700370062cabf008080fb00b0ff2f0033
:10e7e40000806000e80f500001003a00220007009a
:10e7f4000080fa00000006000000fa0000418000da
:10e804009040900000c8b30000c060000004e00025
:10e8140003003200014180000040eb00904098006a
:10e824000040eb005ceab7000040eb005deab70093
:10e834000000eb00b04088000040eb0014e8b70093
:10e844009a0007007e0b0700c80107000080fa0049
:10e85400000006000000fa005dcabf00e24f50004d
:10e8640002003a0077020700010037003700070072
:10e874000080fa00000006000200fa000041800057
:10e88400104090000080fb004600de006140600004
:10e89400004f7800018220000082200010407800a0
:10e8a4008048780010c8bf00e84f50000c003a00c0
:10e8b40000802000204090000080fb00b0248800ed
:10e8c400b02480000000e0000300320000c1b30067
:10e8d40010e8b7000200370040c0b30010e8b700ea
:10e8e4005dcabf00e14f500015003a0000418000ae
:10e8f40081802000110098000b0207005ccabf0051
:10e90400e24f500004003a000141800040c8b300c7
:10e91400904098000b0037001e04e00004003a0009
:10e924000141800080ccb30090409800050037007e
:10e934000141800080c8b300904098000100370076
:10e94400020007000080fa00000006000400fa003c
:10e954005dcabf00e24f50002e003a0094c4bf00cd
:10e964000042b2000004e0002a003200a0528000fd
:10e9740010407800e84f500026003a00a052800072
:10e9840010409000c2c3b3008240600040c3b30093
:10e9940080cf50001f003a00b05280009040900099
:10e9a40000c8b30000c060000004e00019003a0091
:10e9b400b052800001802000110098000040eb005c
:10e9c400204798000f0037002e4090000080fb0085
:10e9d4008000780000802000008140002e409000dc
:10e9e4000080fb00800078008080200000804000d0
:10e9f40010407800004978002e4090000040e80064
:10ea0400204798002e409000e74f5000eeff36005c
:10ea1400130037000040eb005deab700b1528000fc
:10ea240080c0b30080487800b1528000008020008c
:10ea340090009800b1528000c0c8b3009040980084
:10ea4400014180000040eb009040980000418000ac
:10ea5400000f78009e0078000040eb009040980082
:10ea64008081200090009000000820000080600059
:10ea74000000e0000b003200808120003000900094
:10ea84000000e0000300320080812000300090008c
:10ea94000000010081812000110090000070a1009d
:10eaa400900098000080fa00000006000400fa00bc
:10eab40000802000104078000046b2000004e0000e
:10eac40043003a0000802000104090000080fb00ca
:10ead4006101b900028fbe00b000200001002000d7
:10eae4001e01be00800f5100818f590038003e0086
:10eaf4001e00be00006001001a0037001b00370032
:10eb040033003700190037003100370006003700a2
:10eb1400090037002d0037000b00370008003700cc
:10eb2400140037001f00370014e8a80080c0b300a9
:10eb340010e8b700260037008a00070024003700d9
:10eb44000d02070022003700108120009040880049
:10eb54001408a80010c0b30016e8b70014e8a80011
:10eb64001b003700ba000700190037001a0007001d
:10eb74001700370000802000404090000080fb0018
:10eb84008000780020a5200000804000904088008c
:10eb94001408a80010c0b30016e8b70014e8a800d1
:10eba4000b00370014e8a8000080200040409000cb
:10ebb4000081fb0000802000a040900020a52000e0
:10ebc400000041000148780001003700a00a070056
:10ebd4000080fa00000006000600fa000080200011
:10ebe40020409000e14f50000f003a0000802000c8
:10ebf400104078007f4060000004e0000a003a0002
:10ec040014e8a8000080200010409000e34f50005a
:10ec140003003a001000200000538800020037006f
:10ec24000000eb000053880000802000204090008a
:10ec34000004e00049003a00008020001040780001
:10ec44007f406000e24f500044003a000080200002
:10ec5400404090006f4060000004e0003f0032003c
:10ec640014e8a8000040eb00004f7800380037009b
:10ec740000202100200798000080200040409000e0
:10ec84006f4060000080fb000000400080007800be
:10ec940000802000404090000080fb004700de0020
:10eca4000080fb00008040004200dd00800078000e
:10ecb4002e009000010040002007980000802000f2
:10ecc40010409000e34f500004003a00ae00900062
:10ecd40040c8b300904098001c003700008020001a
:10ece400404090006f4060000080fb000000400046
:10ecf40080007800a04a200000804000100798009f
:10ed04001e00900090007800d0ff2f0080806000eb
:10ed14001e0090000108780000802000c040900090
:10ed240000c8b30000c060000004e000040032002a
:10ed3400ae00900000c4b300904098000300370078
:10ed4400ae00900080ccb300904098001e4fe800c5
:10ed540010c0b3009e4f1000c5ff36000080fa00bb
:10ed6400000006000200fa000080200090407800b5
:10ed740000c8b30080cf500033003a0000ccb30089
:10ed840014e8b70000802000304090000080fb00b1
:10ed9400000f78001e007800e20f50000c003200d3
:10eda4001e007800e30f5000170032001e007800a8
:10edb400e10f5000010032002100370000762900e5
:10edc4009040880020012000b04088001e003700d9
:10edd40000802000204090000080fb0000004000e4
:10ede40080007800408029000080400010007800f6
:10edf40090408800904080000080e8001000780077
:10ee0400b0408800100037000080200020409000af
:10ee14000080fb0000004000800078006080290032
:10ee240000804000100078009040880090408000ee
:10ee3400104078000080fb00b040880002003700da
:10ee44000040eb0014e8b7000080fa000000060060
:10ee54000400fa000040eb0008e8b7000040eb00b3
:10ee640009e8b70000802000904078007fc060006f
:10ee74000080fb00100798001e009000e10f500076
:10ee8400120032009e009000e28f50001100320008
:10ee94001e0090000000e00001003200270037004f
:10eea40014e8a80008c8bf000004a00008e8b700e0
:10eeb40000538000e10f500020003a0008c8bf0052
:10eec4000014a00008e8b7001c00370014e8a800ec
:10eed4001a00370014e8a80000202100000f780071
:10eee40000802000404090006f4060000080fb00e4
:10eef4000000400080007800008020004040900026
:10ef04000080fb004700de000080fb000080400022
:10ef14004200dd001e0f40001e00780010409000eb
:10ef24000080fb004200de00610060000004e0009d
:10ef34000200320010c0b30008e8b700a04080000f
:10ef440001082000010060000000e000050032001c
:10ef540080802000904088001408a80020c0b300de
:10ef640016e8b7000080fa00000006000000fa006e
:10ef740094a4a900a04080000108200001006000c2
:10ef84000000e00025003a008081200090009000fd
:10ef940000082000008060000000e0001200320041
:10efa40020c0b3005deab700014180000040eb00df
:10efb400804878000141800080ccb30090409800e4
:10efc400b152800080c0b30080487800b152800004
:10efd4008080200090009800b152800080ccb30063
:10efe400904098004e003700b152800080c0b300ba
:10eff40080487800b1528000008020009000980082
:10f00400b1528000c0c8b300904098000141800014
:10f0140040c8b30090409800410037008081200030
:10f024009000900000082000008060000000e000d4
:10f034003b003a00008020009040780000c8b300f4
:10f0440000c060000004e0002400320000802000c2
:10f05400b0009000b0408000808f50000300310069
:10f064000080200030009000b04088002e0007008f
:10f0740010c0b3005deab700b152800080c0b30095
:10f0840080487800b15280000080200090009800f1
:10f09400b152800000c8b30090409800a152800093
:10f0a40080c0b30080487800a15280000080200016
:10f0b40090009800a152800000c8b30090409800ce
:10f0c4000141800080802000900098000141800070
:10f0d40080ccb300904098001100370020c0b300ea
:10f0e4005deab700014180000040eb0080487800f1
:10f0f4000141800080ccb30090409800b152800060
:10f1040080c0b30080487800b15280008080200025
:10f1140090009800b152800080ccb30090409800d9
:10f124000080fa00000006000200fa00b0408000ef
:10f13400e70f50000e003e00b0408000000f780042
:10f144005ccabf000004e00003003a0010c0b30032
:10f154005ceab700080037005ccabf00e14f50000a
:10f1640005003a0020c0b3005ceab7000200370093
:10f1740080002000000f78000241800000418000e0
:10f18400904090001e40900000c070001041980014
:10f19400014180001e40780080487800b140800022
:10f1a4001e00780000805000b0408800808020005d
:10f1b400f0528800a0408000610060000000e00080
:10f1c4001b003a000b003700f1528000924080008f
:10f1d40012407800804878000100e800f05288006e
:10f1e4000200e800904088001e0078000000e9005a
:10f1f400000f78001e0078000000e000f2ff3a00e3
:10f204000e003700f15280009240800012407800d6
:10f21400804878000100e800f05288000200e8000d
:10f22400904088001e0078000000e900000f78007c
:10f234001e0078000000e000f2ff3a000080fa00af
:10f24400000006000200fa00a052800090407800fe
:10f25400114798001e4090008080fb0080812000b0
:10f2640020009000808f5000040036008081200030
:10f27400200090001047980007003700808120008c
:10f28400a00090001e4090000080fb008080500091
:10f2940080812000210098000040eb00004f78009e
:10f2a4000b00370080812000100178009e80fb0055
:10f2b40080802000008040001040780000497800e1
:10f2c4008200e80080812000010878001e4fe800d9
:10f2d4001e4090009e4f1000f2ff390080812000f4
:10f2e400200090000000e00013003200b1528000c2
:10f2f40080c0b30080487800b15280008080200034
:10f3040090009800a0528000104090000044b20089
:10f314000004e00004003a00b152800080ccb30045
:10f324009040980012003700b152800080c8b300aa
:10f33400904098000e003700b152800000802000f9
:10f344009000980080812000300090000000e000d0
:10f354000300320080812000300090000000010092
:10f3640081812000110090000070a100900098009d
:10f374000080fa00000006000000fa0014e8a8006b
:10f384000040eb0052eab7000080200020409000cb
:10f3940011e8b70000802000204090000004e00045
:10f3a40003003a0000c1b30010e8b70003003700bf
:10f3b40000c2b30010e8b700a80807000080fa00f4
:10f3c400000006000400fa00204798003147980026
:10f3d40000202100000f78002e4090000080fb00e8
:10f3e40000004000800078003e4090000080fb0058
:10f3f400008040004200dd004200de004200dd00eb
:10f404001e0f40009e007800114090000070a10083
:10f41400904098003e4090000004e00007003a004d
:10f424002e4090000080fb008000400080a520005a
:10f43400008040001e087800060037002e4090002f
:10f444000080fb008000400000822000008040001b
:10f454001e0878009e007800114090000060a00013
:10f46400904098000080fa00000006000400fa00b2
:10f4740020479800314798002e4090000080fb0000
:10f484000000400080007800a04a20000080400076
:10f49400000f78003e4090008080fb001e00780042
:10f4a400010878003e4090000080fb004300de002d
:10f4b400610060000004e000030032008040eb00c3
:10f4c4002e409000bfff07003e4090000080fb00ec
:10f4d4004200de00610060000004e000030032002e
:10f4e40011c0b3002e409000b6ff07000080fa0060
:10f4f400000006000400fa002047980031479800f5
:10f504002e4090000004e0000d003a00b15280004b
:10f5140080c0b30080487800b15280000080200091
:10f5240090009800b1528000c0c8b3009040980089
:10f534000141800040c8b300904098001200370099
:10f544002e4090000080fb00000040008000780006
:10f554003e4090000080fb00008040004200dd003f
:10f56400800078000020210000804000000f780017
:10f574001e0078009040900040c8b30080c0700026
:10f584001e007800114098000080fa000000060078
:10f594000800fa0020479800314798002207980095
:10f5a400634798003e4090000004e00007003200ea
:10f5b4002e4090000080fb0080004000008220006c
:10f5c40000804000100f7800060037002e409000a5
:10f5d4000080fb008000400080a5200000804000e7
:10f5e400100f78001e0078009040900000c4b30013
:10f5f40080c068001e007800114098001e0078004a
:10f60400ae009000110098001e0078006e4190003a
:10f61400024878001e0078001040900002c4b30035
:10f62400824060001e007800114098001e0078009f
:10f634009040900080c8b30080c070001e00780025
:10f64400114098003e4090000004e0001000320099
:10f654002e4090000080fb000000400080007800f5
:10f664000082200000804000000178002e409000bd
:10f674000080fb0000004000800078000082200031
:10f684000080400010407800004978000f003700e7
:10f694002e4090000080fb000000400080007800b5
:10f6a40080a5200000804000000178002e409000da
:10f6b4000080fb00000040008000780080a520004e
:10f6c4000080400010407800004978001e00780057
:10f6d4000080fa00000006000400fa00000f780021
:10f6e400214798002e4090008080fb0010002000ed
:10f6f4000100dd00804078001e0078000148780099
:10f704000080fa00000006000000fa000000eb0090
:10f71400208288004282200003c4b3008040eb00b2
:10f7240010c0b3009aff0700108288000040eb006d
:10f734000af0b7006000b800508288006182880037
:10f744006000b80070828800818288000000eb00ad
:10f75400408288000040eb0019f0b7001400370025
:10f7640050838000000001000004e0000c0032001f
:10f7740020838000000001000004e0000800320043
:10f7840019d0bf008080fb00100020000100dd00c4
:10f7940080007800408280000080700040828800f1
:10f7a400af03070019d0bf000040e80019f0b7000c
:10f7b40019d0bf000004e000e9ff32000080fa0025
:10f7c400000006000000fa000080200010407800cd
:10f7d4007f406000e14f500013003a000080200099
:10f7e400404090000004e0000f003a000080200038
:10f7f400104090008080fb00e00f2000808f5000bc
:10f8040001003200080037000040eb0008e8b700b0
:10f81400808020009040880010002000b0408800c4
:10f8240010ccb30014e8b7000080fa000000060012
:10f834000400fa000ad0bf000080fb001007980003
:10f844001e009000e10f50006d0032001e00900079
:10f85400e10f500004003c001e0090000000e00096
:10f86400080032009c0037001e009000e20f500098
:10f87400690032001e009000e30f50007600320051
:10f8840095003700108280000000e000060032007e
:10f89400108280009040900000c8b30000c0600057
:10f8a4000004e0008c003a002041800031418000d7
:10f8b4006080880071808800404180005141800050
:10f8c40080808800918088006041800071418000c0
:10f8d400a0808800b180880030c8bf0018f0b7004d
:10f8e40031c8bf0019f0b70032c8bf001af0b70022
:10f8f4000040eb00004f78000a0037001e81fb0037
:10f904001e80fb00ee00400040822000008040008a
:10f9140090409000a0012100000041001140980097
:10f924001e4fe80032c8bf009e4f5000f3ff3e0058
:10f9340010828000104078002cf0b7002cd0bf005b
:10f94400ff4f500064003a006280800073808000a2
:10f954005035250021342400800f5100818f590037
:10f964005d003a0019d0bf00ef4f50005a003e002e
:10f974001ad0bf00f04f500057003e001ad0bf000d
:10f984000004e0005400320018d0bf000004e0007e
:10f9940005003200810121009140780000c8b300c5
:10f9a40080cf50004c003a0080808000918080001d
:10f9b40040428800514288005035250021342500fa
:10f9c4002042880031428800810121009140780062
:10f9d40000c8b30080cf500003003a0010c0b30049
:10f9e4000af0b7003c00370018d0bf000004e00064
:10f9f40039003a0020c0b3000af0b70036003700df
:10fa0400ac010700e14f400033003a0030c0b300be
:10fa14000af0b70030003700a6010700e14f4000ac
:10fa24002d003a0050c8bf000004e00007003a006f
:10fa34006042800071428000e00f5000e08f580067
:10fa44000200320020c0b30050e8b70030c0b30059
:10fa54000af0b70020003700208280000000e00098
:10fa640006003200208280009040900000c8b3005d
:10fa740000c060000004e00017003a004284200047
:10fa8400d3c0b30011c0b30010c0b300c0fe070060
:10fa940020828800108280000000e000060032000e
:10faa400108280009040900000c8b30000c0600045
:10fab4000004e00006003a004282200003c2b300c2
:10fac4008040eb0010c0b300b1fe07001082880034
:10fad4000040eb000af0b7000ad0bf000080fb0032
:10fae4000080fa00000006000c00fa0078d0bf0085
:10faf4000080fb00500798005e009000fe0f50004d
:10fb04009e003200de009000fe8f500014003c0086
:10fb14005e009000f20f500032003200de009000d0
:10fb2400f28f500007003c005e0090000000e000ef
:10fb3400a9003200de009000e38f5000650032001f
:10fb4400d50037005e009000fa0f50007a003200b2
:10fb5400de009000fb8f5000b0003200ce00370072
:10fb6400a0022000de009000808f5000530032007d
:10fb7400a0022000de009000808f500009003c00ad
:10fb840050022000de009000808f500023003200dd
:10fb940080022000de009000808f5000410032007f
:10fba400bd003700d00f2000de009000808f500091
:10fbb400a2003200f00f2000de009000808f500081
:10fbc40005003200f0022000de009000808f50001b
:10fbd40092003200b00037001bd0bf0078f0b700ad
:10fbe400bd00370060892900218520002300090019
:10fbf400b05878004002b10040022000010020000b
:10fc040060428800714288000040eb0050e8b70071
:10fc1400d0cfb30078f0b700af0037000040eb005e
:10fc240050e8b700308380000000010030079800de
:10fc3400410798004083800000000100010020007b
:10fc440010079800210798001e48900052e8b7005a
:10fc54000e48900053e8b7007e40900054e8b70087
:10fc64006e40900055e8b7005e40900056e8b7003b
:10fc74004e40900057e8b7003e40900058e8b70067
:10fc84002e40900059e8b7008000200001002000b9
:10fc94006042880071428800d0cfb30078f0b7008a
:10fca4008d0037003b0107000004e0008a003a00a1
:10fcb40000c0eb0078f0b70087003700cf010700e1
:10fcc4000004e00084003a0000c0eb0078f0b700c4
:10fcd400810037000040eb00004f78000a00370035
:10fce4001e81fb009e80fb00d002210000804000aa
:10fcf40010407800804078002085200000004100fa
:10fd0400014878001e4fe80010c1b3009e4f100058
:10fd1400f3ff36002001200001002000604288002b
:10fd2400714288000040eb0050e8b700d0cfb30028
:10fd340078f0b7006800370020c0b30052e8b7007d
:10fd44000040eb0053e8b7000040eb0054e8b70074
:10fd54000040eb0055e8b7000040eb0050e8b70066
:10fd640040002000010020006042880071428800a9
:10fd7400d0cfb30078f0b70057003700508380002d
:10fd8400000001000004e000060032000040eb0027
:10fd940050e8b7006000b8006042880071428800f3
:10fda4000a0037002f10a9002f30a8002f50a900f7
:10fdb4002f70a900a0c3b30039f0b7000040eb00d6
:10fdc4003af0b70010c0b30050e8b70000c0eb0031
:10fdd40078f0b700400037002fd0bf006f406000bc
:10fde400e64f500006003a0050c8bf00e14f5000f3
:10fdf40003003a0000c0eb0078f0b700360037008b
:10fe0400170207006000b800604288007142880051
:10fe140000c0eb0078f0b7002f0037000040eb0083
:10fe240050e8b7006000b800604288007142880062
:10fe340000c0eb0078f0b700270037002082800074
:10fe44000000e00006003200208280009040900014
:10fe540000c8b30000c060000004e0001e003a00c7
:10fe64006042800071428000228520008041780039
:10fe740011c0b30010c0b300c5fd07002082880084
:10fe840000c0eb0078f0b7006000b8006042880062
:10fe94007142880010003700f10107002f10a800fc
:10fea4002f30a9002f50a8002f70a90000c2b30062
:10feb40039f0b7000040eb003af0b70010c0b300cf
:10fec40050e8b7006000b8006042880071428800c2
:10fed400d0cfb30078f0b7000080fa00000006002d
:10fee4000400fa0078d0bf000080fb0010079800df
:10fef4001e009000f20f50003d0032009e00900062
:10ff0400f28f500007003c001e0090000000e0004b
:10ff1400320032009e009000e38f50000d0032004a
:10ff24005b003700d00f20009e009000808f5000af
:10ff340040003200f00f20009e009000808f50009f
:10ff4400390032001e009000fe0f500023003200e2
:10ff54004f003700c20107002f10a9002f30a8005e
:10ff64002f50a9002f70a900a0c3b30039f0b70027
:10ff74000040eb003af0b7000040eb00004f78007f
:10ff84000a0037001e81fb009e80fb00d002210086
:10ff940000804000104078008040780020852000d8
:10ffa40000004100014878001e4fe80011c1b30071
:10ffb4009ecf1000f3ff3600200120000100200036
:10ffc40060428800714288000040eb0050e8b700ae
:10ffd400d0cfb30078f0b7003400370010c0b300be
:10ffe40050e8b70000c0eb0078f0b7002f003700ee
:10fff400608929002185200023000900b058780079
:020000040001f9
:100004004002b1004002200001002000604288004c
:10001400714288000040eb0050e8b700d0cfb30035
:1000240078f0b700210037001bd0bf0078f0b7008c
:100034001e003700208280000000e000060032002d
:10004400208280009040900000c8b30000c060008f
:100054000004e00015003a00604280007142800014
:10006400228520008041780011c0b30010c0b30085
:1000740047fd07002082880000c0eb0078f0b7003d
:100084006000b800604288007142880007003700b1
:1000940011c0b30010c0b30016fd070010c0b300b8
:1000a40050e8b70000c0eb0078f0b7000080fa0019
:1000b400000006000000fa005083800000000100e8
:1000c4000004e0000b003a0019d0bf008080fb0060
:1000d400100020000100dd000080ea0080007800ac
:1000e4004082800000806000408288007cff07001e
:1000f4002400370019d0bf008080fb0010002000ce
:100104000100dd00800078004082800000806000f3
:100114000000e0001a003a00208380000000010083
:100124000004e0001400320019d0bf008080fb00fe
:10013400100020000100dd00800078004082800073
:1001440000807000408288002f10a9002f30a80082
:100154002f50a8002f70a90080c2b30039f0b70057
:100164000040eb003af0b70010c0b30050e8b7000d
:100174005dfe07000300370059ff07000100370048
:1001840059fe070078d0bf000080fb000080fa0011
:10019400000006000200fa0002d0bf000080fb004d
:1001a400000f78001e007800e20f50002f0032008c
:1001b4001e007800e20f500007003c001e0078008b
:1001c4000000e0000b0032001e007800e10f500038
:1001d4001b003200850037001e007800e30f50003a
:1001e4004a0032001e007800e40f50005100320033
:1001f4007e0037001dd0bf0009f0b7001ed0bf003d
:1002040008f0b7001fd0bf0007f0b70020d0bf0030
:1002140006f0b70022d0bf0005f0b70023d0bf001e
:1002240004f0b7000040eb0050e8b7006000b800ed
:10023400604288007142880010c0b30002f0b70029
:10024400208080000000e00003003a000040eb0042
:1002540002f0b70065003700208080000000e9004c
:100264002080880020c0b30002f0b7002082800004
:100274000000e000060032002082800090409000e0
:1002840000c8b30000c060000004e00057003a005a
:1002940063838000228520003080800041808000bc
:1002a40003000100e14f50000800320010c0b30009
:1002b40050e8b7006000b8006042880071428800ce
:1002c40010c0b3000af0b700480037003080800047
:1002d4004180800061004000e08048003080880058
:1002e400418088000040eb0050e8b7000020200067
:1002f40001002000604288007142880020852000af
:100304000082880030c0b30002f0b7006042800071
:1003140071428000e00f5000e08f580003003a0063
:1003240010c0b30002f0b7003000370040c0b30083
:1003340002f0b70050c8bf000004e0002b003a00f0
:100344006242800073428000f0032000010020001c
:10035400800f5100818f59002400360020828000d4
:100364000000e000060032002082800090409000ef
:1003740000c8b30000c060000004e0001b003a00a5
:100384000282800003c4b30011c0b30010c0b300e4
:100394007ffc07002082880030c0b30002f0b70061
:1003a400a2808000b380800000fc2f00f1ff2f00aa
:1003b4000200400083804800a0808800b18088004b
:1003c400624280007342800000fc2f00f1ff2f0086
:1003d4000200400083804800604288007142880027
:1003e400008280000004b0000082880002d0bf00b8
:1003f4000080fb000080fa00000006000200fa0002
:1004040003d0bf000080fb00000f78001e007800be
:10041400e20f50007b0032001e007800e20f500013
:1004240007003c001e0078000000e0000b003200d2
:100434001e007800e10f50001800320084003700dd
:100444001e007800e30f5000220032001e007800e6
:10045400e40f5000480032007d0037001dd0bf007b
:1004640009f0b7001ed0bf0008f0b7001fd0bf00ce
:1004740007f0b70020d0bf0006f0b70022d0bf00bd
:1004840005f0b70023d0bf0004f0b7000040eb0034
:1004940050e8b70010c0b3000af0b7002080800015
:1004a4000000e00003003a000040eb0003f0b70056
:1004b4006700370030c0b30003f0b7002085200088
:1004c4000082880000202000010020006042880093
:1004d400714288006042800071428000e00f500049
:1004e400e08f580012003200108280000000e0000b
:1004f40006003200108280009040900000c8b300d3
:1005040000c060000004e00051003a000282800054
:1005140003c4b3008040eb0010c0b3001cfc070010
:100524001082880040c0b30003f0b7001200370007
:1005340070838000000001000004e0000b00320022
:100544002f10a9002f30a8002f50a9002f70a90048
:1005540070c2b30039f0b7000040eb003af0b700c6
:1005640010c0b30050e8b7003900370020c0b30012
:1005740003f0b70036003700108280000000e0006e
:1005840006003200108280009040900000c8b30042
:1005940000c060000004e0002d003a00a28080004a
:1005a400b380800010828000104078000080fb003f
:1005b400010020000000510081805900a0808800c3
:1005c400b180880062428000734280001082800003
:1005d400104078000080fb00010020000000510062
:1005e4008180590060428800714288000082800046
:1005f4000004b0000082880030c0b30003f0b700ec
:10060400130037008483800022852000308080001e
:10061400418080008041eb0004000100e14f500064
:100624000b003a003080800041808000610040006f
:10063400e08048003080880041808800208080006d
:100644000000e9002080880010c0b30003f0b70068
:1006540003d0bf000080fb000080fa000000060009
:100664000000fa00d10221009140780000c8b300d4
:1006740000c0600001c7b300014070002df0b70056
:100684002df0a9000040eb002ef0b7002f10a900b8
:100694002f30a9002f50a9002f70a9002fb0a90056
:1006a4002fd0a9002ff0a9000040eb0030f0b700d4
:1006b4000040eb0031f0b7000040eb0032f0b7002f
:1006c4000040eb0033f0b700a0c0b30034f0b70033
:1006d40035d0bf006040600035f0b70036d0bf00b1
:1006e4006040600036f0b70037d0bf006040600063
:1006f40037f0b70038d0bf006040600038f0b70072
:100704000040eb0039f0b7000040eb003af0b700ce
:100714000040eb003bf0b7000040eb003cf0b700ba
:100724000040eb003df0b7000040eb003ef0b700a6
:100734000080fa00000006000000fa00eac2bf00d0
:100744000004a2000080fb00610060000080fa0049
:10075400000006000000fa00002020000080fa00db
:10076400000006000000fa0090838000a18380004e
:100774000080fa00000006000000fa00e802a80069
:10078400ca22a800c822a900e822a8000080fa0012
:10079400000006001200fa0010c0b30020479800c1
:1007a40030002000000f7800ca22a8000000eb00ef
:1007b4001012880000052000200798002e009000e9
:1007c4000000e00020003a0010128000f103200035
:1007d40001007000101288001b0037002e009000ea
:1007e400e80f50000c0036001e0fe9002e009000a8
:1007f400630060000000e000030032002e0090005f
:1008040064004000200798002e0090004200de00a3
:10081400200798000c0037002e0090004200dd00f5
:100824000080ea007c0060009e00700010128000ce
:100834008080700000022000008070001012880088
:100844000000eb00200798002e0090000000e0005c
:10085400e2ff3a000041eb0031c0b3000002200087
:100864008d02070010c0b3005f0207000000eb0018
:10087400200798000500370000c0eb00b70207000e
:100884002e0090000000e800200798002e00900041
:10089400e90f5000f8ff3600ca22a90010c0b300c7
:1008a40051020700680047006011b8008040eb0067
:1008b400600007004e009000300798006e409000e2
:1008c400e14f4000060032006e4090008080fb0043
:1008d400700f200000806000e10f5000070032001c
:1008e4000040eb0020479800ca22a8002e40900048
:1008f4000080fb00000f980046003700f0ff200046
:10090400200798006a0047006011b80011c0b300c6
:10091400480007005e009000300798002e00900009
:100924000000e900200798006e4090000004e000f9
:10093400030032002e0090000000e000f1ff3a00b6
:100944002e0090000000e00004003a000040eb009c
:1009540020479800ca22a8002b00370020c0b3000b
:10096400210207000041eb0031c0b300e003200086
:100974004902070011128000b003200000807000bb
:10098400101288006c0047006011b80061c1b30008
:10099400280007006e009000300798006e004700a2
:1009a400022020000300200061c0b30021000700e2
:1009b4007e00900030079800f00f20002007980078
:1009c400030037002e0090000000e9002007980083
:1009d4002e0090000000e000050032000001eb0052
:1009e4006000b800a2000700e14f5000f5ff3a0094
:1009f4002e0090000000e00003003a000040eb00ed
:100a040020479800ca22a8002e4090000080fb00d6
:100a1400000f98000e0890000080fa000000060005
:100a24000000fa0015020700ca22a8000080fa009c
:100a3400000006001600fa00200f9800614f98008d
:100a4400020f9800130f98008000200010079800f0
:100a5400ca22a9006e4890000080fb00c2802900d1
:100a64006600b9000200400090407800660047002c
:100a740061409800660047000e0990009e099000ae
:100a840012009800230098006e4890000080fb003c
:100a9400c28029006600b900020040009040900026
:100aa4006600470001487800e600470031009000e6
:100ab4000060a000b000980066004700604090000d
:100ac40026020700660047005040900023020700fa
:100ad400660047004040900020020700660047007f
:100ae400304090001d02070066004700204090003f
:100af4001a0207006600470010407800170207003a
:100b04006e4890000080fb00c28029006600b90096
:100b14000080e800600079000000e0000800320076
:100b24006e4890000080fb00c28029006600b90076
:100b34000080e80060007900e10f50000c003a00ea
:100b4400c3010700404798001e0090000000e90020
:100b5400100798004e409000e14f400011003a0009
:100b64001e0090000000e000f5ff3a000d00370081
:100b74006e4890000080fb00c28029006600b90026
:100b84000080e80060007900e20f500005003a00a0
:100b9400af010700ae01070050479800ac01070001
:100ba400404798006e4890000080fb00c2802900f6
:100bb4006600b9000080e80060007900e10f500091
:100bc40019003a000040eb00404798000040eb0059
:100bd400004f78000e0037000080eb0010079800eb
:100be4009b010700404798001e0090000000e900a8
:100bf400100798004e4090000004e00003003a0003
:100c04001e0090000000e000f5ff3a001e4fe800cf
:100c140080c1eb009ecf1100030032004e409000d3
:100c24000004e000ecff320000c0eb00cb01070041
:100c34006e4890000080fb00c28029006600b90065
:100c44006400400002004000104078000004e0000e
:100c540001003a00ca22a800ae0090002e089000bd
:100c6400010878002e0890000080fa0000000600b9
:100c74002000fa00200f9800310f9800420f9800ce
:100c840010c0b300404f98002e089000be0890009a
:100c94004909dd00c700de00810071004900dd0064
:100ca40040079800510798007a0047004e019000d1
:100cb400de01900071c0b3005eff07005e08900083
:100cc400100f98002e5090000004e0000d00320038
:100cd4007c0047004e019000de01900071c0b3001b
:100ce40054ff07006e089000100f98002e509000db
:100cf4000004e000030032008001eb00730f980051
:100d0400c7003700f02f2000000f980000042000d7
:100d140070079800030037007e0090000000e9008f
:100d2400700798007e0090000000e000faff3a008f
:100d340047010700504f98000e0890000000e9009a
:100d4400000f98000004200070079800030037008b
:100d54007e0090000000e900700798007e0090007b
:100d64000000e000faff3a005e489000e14f4000c6
:100d740003003a000e0890000000e000ecff3a0087
:100d84000e0890000000e000030032005e4890006e
:100d9400e24f4000030032000040eb00404f980057
:100da400990037002e089000be089000e00f500014
:100db400e08f580006003a004e0890000000e00062
:100dc40003003a006000b80090838800a183880083
:100dd4000000eb00000f9800830037004e089000dd
:100de4000000e0000c003200f00f200040128800e8
:100df40040c2bf00614060000004e000fcff32001c
:100e04008e0890004e0890008080400040128000c0
:100e140080487800710037002e089000be089000ca
:100e2400e00f5000e08f58006b003a008e089000ed
:100e3400601c2000808f50000c0032008e0890004f
:100e4400601d2000808f5000080032008e08900042
:100e5400601e2000808f5000040032008e08900035
:100e6400601f2000808f500059003a00f8000700ee
:100e74000080fb0001002000200798003107980043
:100e8400f30007000080fb00010020004809dd009a
:100e9400c801de00830171004801dd002e009000ce
:100ea400be0090000200700083807000200798004c
:100eb40031079800e60007000080fb0001002000d5
:100ec400c001dd00020020002e009000be00900052
:100ed400020070008380700020079800310798009a
:100ee400db0007000080fb0001002000c801dd00da
:100ef400020020002e009000be009000020070004e
:100f0400838070002007980031079800d000070004
:100f14000080fb0001002000008fbe00cc00070011
:100f24000080fb0001002000c808dd000080fd00f7
:100f3400804078000040eb001e1f70001e97700078
:100f4400c30007000080fb0001002000c000dd009a
:100f5400000020001e1f70001e977000bc000700d8
:100f64000080fb0001002000c800dd00000020001c
:100f74001e1f70001e9770000e089000680040004d
:100f8400000f98002e009000be0090003e0140002b
:100f9400ae81480090838000a1838000800f5100bf
:100fa400818f59000d0036002e009000be00900085
:100fb4003e014000ae8148000200be0061005000c6
:100fc400e080580090838800a183880003003700e4
:100fd4009f000700010037009d0007000e089000e5
:100fe4000000e800000f98008e089000f01f200019
:100ff400808f500079ff360000c0eb00d700070057
:1010040000c0eb00d500070000c0eb00d3000700d0
:10101400ca22a8004e4890000080fb00700f980080
:101024007e0890000080fa00000006001000fa001c
:10103400300798004107980052079800434f9800e2
:1010440010c0b300004f78003e009000ce00900026
:10105400e00f5000e08f580006003a004e48900020
:101064000004e00003003a000040eb00004f780069
:10107400520037003e009000ce0090004909dd0088
:10108400c701de00830171004901dd006e004700e5
:1010940091c0b30067fe07007e009000200798000f
:1010a4004e4090000004e000030032000040eb00da
:1010b400004f780040003700e0cfb300a7000700de
:1010c4000000eb00100798000f0037009e0090000e
:1010d4005e00900000804000104078000080fb001b
:1010e4004012880040c2bf00614060000004e0007c
:1010f400fcff320040128000104798001e00900050
:101104000000e800100798009e009000f01f2000e7
:10111400808f5000edff360000c0eb008f00070009
:1011240000c0eb008d00070049000700104798003d
:101134001e4090000080fb006f006000e50f50002f
:10114400030032000040eb00004f78001800370025
:101154000000eb0010079800f00f200040128800f8
:1011640040c2bf00614060000004e000fcff3200a8
:1011740040128000104798001e0090000000e80014
:10118400100798001e4090000004e00003003a009d
:101194001e0090000000e000efff3a001e009000e7
:1011a4000000e00002003a000040eb00004f78002d
:1011b40000c0eb0069000700ca22a8001e80fb00e3
:1011c4000080fa00000006000000fa00eac2bf0036
:1011d4000080fb000000d100614060000080fb0043
:1011e4000080fa00000006000800fa00604798003a
:1011f4006e409000404798000c003700b07c2000ff
:1012040001002000008fbe000080eb008080eb0016
:101214001e0f40005e9748000080eb008080eb00ca
:10122400be0f1000ae8f1800f7ff3a004e4090003a
:101234000040e900404798004e409000e14f4000d4
:10124400eeff3a00000000000080fa0000000600f3
:101254000000fa00f00f20004012880040c2bf00d6
:10126400614060000004e000fcff32004012800096
:101274000080fb000080fa00000006000000fa0075
:1012840000128000f1ff27000100600000128800b6
:101294000080fa00000006000800fa00000f780041
:1012a40021479800324798000000eb0000128800a4
:1012b4003e4090008080fb0010128000008070008f
:1012c400101288002e4090000080fb002007980038
:1012d4002e009000e20f5000090032002e00900012
:1012e400e30f5000080032002e0090000000e000e0
:1012f40001003200060037004302a8000400370052
:1013040042c2a8000200370042c2a8004302a9005a
:101314001e007800300798003e009000e40f500053
:10132400040032003e009000e50f5000020032003d
:1013340004003700c822a800c802a8004322a9005c
:1013440001003700c802a900e902a900d842a80098
:1013540041e2a8000080fa00000006000400fa0040
:10136400204798002e4090000080fb004012880027
:1013740040c2bf00614060000004e000fcff320096
:1013840040128000004f78000000eb000080fa005b
:10139400000006000a00fa006800470030079800c1
:1013a4005c0007008ac70700100798002ca3a90057
:1013b40023c3bf007f40600023e3b70000c0eb00fd
:1013c40024e3b70020c3bf007f40600020e3b700e0
:1013d400513220009140780000ceb30000c060007c
:1013e4000044a00025e3b7001132200091407800aa
:1013f400c0cfb30000c0600021e3b7002132200059
:101404009140780030ccb30000c0600022e3b70004
:10141400500020004019880021e3a8002116800014
:10142400c0ff2f0000806000201688000116800095
:10143400c0ff2f000080600000168800c0e2a800f2
:101444000000eb0020079800000037000df40700af
:101454004900070010c8bf00ff4f500003003e00c2
:1014640010c8bf00e14f5000f8ff3e001e0090007e
:10147400e10f500021003a00c2c2bf0001c8b3000e
:10148400014060000004e00013003a002e009000c8
:101494000000e0000a00320043000700004f78001b
:1014a4001e80fb00801f7800a08b2900801f78001d
:1014b4002e00900057ee0700e48757000400370021
:1014c400f18b2900108c2900c7d60700200798004b
:1014d400c402a800ddff37002e0090000000e000e9
:1014e400040032002e00900052d207000000eb00ee
:1014f40020079800c402a900d4ff37008efc07001f
:10150400e14f5000d1ff3a0031c70700100798009f
:10151400ceff37000000fa000080eb00601988005d
:10152400816a20009140780000ccb30000c06000c4
:101534007041b300a8e6b700f16c20009140780038
:1015440000ccb30000c060007040b300cfe6b70029
:10155400016c20009140780000ccb30000c0600012
:101564000034a000c0e6b7007480a8008ff3070021
:101574000080fa00000006000000fa0010c8bf0056
:10158400ff4f50000600360088c4bf006240600070
:101594000004e0000100320001003700a4f8070055
:1015a4000080fa00000006000200fa002023a800d0
:1015b4000000eb00000f7800010037001e0fe80068
:1015c400703e20009e0f1000fcff36002023a9006f
:1015d4000000eb00000f7800010037001e0fe80048
:1015e400703e20009e0f1000fcff360020c3bf0099
:1015f400614060000004e000fcff3200001880003d
:101604004200de000080fb000080fa0000000600bb
:101614000000fa000080fa00000006000000fa0052
:101624000080fa00000006000000fa000080fa00c2
:10163400000006000000fa000080fa000000060026
:101644000000fa005ff807000080fa0000000600be
:101654000000fa000080fa00000006000000fa0012
:10166400d1c1b30010c0b30080f7070026f807000b
:101674000080fa00000006000000fa009444a8006c
:1016840080702000b0838800b08380000000e900ef
:10169400b0838800b08380000000e000faff3a00c5
:0c16a4009444a9000080fa000000060039
:020000040000fa
:020000040001f9
:1016b000641000000e00000002000000cc83b400a3
:1016c00083ac83009e833a0086e688001888000079
:1016d0007610000002000000000000000012000070
:1016e0001000000000000000000800006802000078
:1016f000000000007810000002000000020000005e
:10170000ff00000002100000500000000000000078
:1017100072100000040000000000000052100000e1
:101720001200000002000000ffff000000000000a7
:101730000000ff00ffffff000000000000980f0006
:10174000680e00009a01000000000000680a000016
:101750000002000000000000680c00000002000011
:08176000000000000000000081
:020000040000fa
:020000040001f9
:041768000000fe007f
:00000001FF
